:020000040000FA
:100000000C944F010C9477010C9477010C94CE243E
:100010000C94CE240C94CE240C9477010C9477018C
:100020000C9477010C9477010C9477010C94770170
:100030000C9477010C9477010C9477010C94770160
:100040000C9484240C9477010C9452240C942C244A
:100050000C9477010C9477010C9477010C94770140
:100060000C9446250C94770107634236B79BD8A7BA
:100070001A39685618AEBAAB558C1D3CB7CC5763CD
:10008000BD6DEDFD753EF6177231BF000000803F7B
:1000900008000000BE922449123EABAAAA2ABECD97
:1000A000CCCC4C3E00000080BEABAAAAAA3E000009
:1000B0000000BF000000803F000000000008417801
:1000C000D3BB4387D1133D190E3CC3BD4282AD2B38
:1000D0003E68EC8276BED98FE1A93E4C80EFFFBE30
:1000E00001C4FF7F3F00000000004E414E494E49D1
:1000F0005459494E46CDCCCC3D0AD7233C17B7D1F5
:100100003877CC2B329595E6241FB14F0A0000209A
:10011000410000C84200401C4620BCBE4CCA1B0E19
:100120005AAEC59D7400407A10F35A00A0724E1862
:10013000090010A5D4E80000E87648170000E40B99
:1001400054020000CA9A3B000000E1F5050000805F
:10015000969800000040420F000000A086010000B9
:1001600000102700000000E8030000000064000009
:100170000000000A00000000000100000000002C48
:1001800076D888DC674F0823DFC1DFAE59E1B1B70D
:1001900096E5E3E453C63AE651997696E8E6C284DA
:1001A00026EB898C9B62ED407C6FFCEFBC9C9F40F2
:1001B000F2BAA56FA5F490055A2AF75C936B6CF917
:1001C000676DC11BFCE0E40D47FEF520E6B500D0ED
:1001D000ED902E0300943577050080841E08000002
:1001E000204E0A000000C80C333333330F986E12D0
:1001F000831141EF8D2114893BE65516CFFEE6DBD6
:1002000018D1844B381BF77C1D901DA4BBE424201F
:100210003284725E228100C9F124ECA1E53D270001
:100220005EBCE2613FDD83C29C7E20A3FD1F4100D6
:100230009D23BE46DB65F88C11AF32CA57E97400C6
:10024000000000240027002A00000000080002012E
:100250000000030407000000000000000000000090
:100260000023002600290000000000250028002BA4
:10027000000404040404040404020202020202034F
:100280000303030303010204081020408001020459
:10029000081020010204081020007126932B11245D
:1002A0001FBECFEFD8E0DEBFCDBF26E0A0E3B3E0B6
:1002B00001C01D92A931B207E1F713E0A0E0B1E05F
:1002C000E8EEF0E702C005900D92A033B107D9F730
:1002D00011E0CEE4D1E004C02197FE010E94DC349D
:1002E000CD34D107C9F70E9406280C9467380C94C6
:1002F0000000089508950895AF92BF92CF92DF92C3
:10030000EF92FF920F931F93CF93DF936C017B01CA
:100310008B01040F151FEB015E01AE18BF08C0175B
:10032000D10759F06991D601ED91FC910190F081CE
:10033000E02DC6010995892B79F7C501DF91CF9191
:100340001F910F91FF90EF90DF90CF90BF90AF90F3
:100350000895CF93DF93FC014481558160817181C1
:1003600082E794E00E947C01EC0142E050E069E504
:1003700071E082E794E00E947C018C0F9D1FDF9169
:10038000CF910895FC01538D448D252F30E0842FAB
:1003900090E0821B930B541710F0CF9608950197AD
:1003A0000895FC01918D828D981761F0A28DAE0F9A
:1003B000BF2FB11D5D968C91928D9F5F9F73928F21
:1003C00090E008958FEF9FEF0895FC01918D828D4D
:1003D000981731F0828DE80FF11D858D90E008951A
:1003E0008FEF9FEF0895FC01918D228D892F90E072
:1003F000805C9F4F821B91098F739927089582E734
:1004000094E00E94F30121E0892B09F420E0822F7F
:10041000089580E090E0892B29F00E94FF0181116E
:100420000C9400000895FC01A48DA80FB92FB11DF4
:10043000A35ABF4F2C91848D90E001968F7399271A
:10044000848FA689B7892C93A089B1898C918370F8
:1004500080648C93938D848D981306C00288F389F1
:10046000E02D80818F7D80830895EF92FF920F931E
:100470001F93CF93DF93EC0181E0888F9B8D8C8D50
:1004800098131AC0E889F989808185FF15C09FB744
:10049000F894EE89FF896083E889F9898081837007
:1004A000806480839FBF81E090E0DF91CF911F91B6
:1004B0000F91FF90EF900895F62E0B8D10E00F5FD7
:1004C0001F4F0F731127E02E8C8D8E110CC00FB6AD
:1004D00007FCFACFE889F989808185FFF5CFCE0145
:1004E0000E941302F1CFEB8DEC0FFD2FF11DE35AAB
:1004F000FF4FF0829FB7F8940B8FEA89FB898081C8
:100500008062CFCFCF93DF93EC01888D8823B9F041
:10051000AA89BB89E889F9898C9185FD03C080810E
:1005200086FD0DC00FB607FCF7CF8C9185FFF2CF8B
:10053000808185FFEDCFCE010E941302E9CFDF91CC
:10054000CF91089590E0FC01E75BFD4F2491FC0101
:10055000EB57FD4F3491FC01EF58FD4FE491EE2332
:10056000C9F0222339F0233001F1A8F4213019F128
:10057000223029F1F0E0EE0FFF1FE959FD4FA59160
:10058000B4918FB7F894EC91611126C030953E2359
:100590003C938FBF08952730A9F02830C9F024304C
:1005A00049F7809180008F7D03C0809180008F7714
:1005B00080938000DFCF84B58F7784BDDBCF84B597
:1005C0008F7DFBCF8091B0008F778093B000D2CF2A
:1005D0008091B0008F7DF9CF3E2BDACFCF93DF93A0
:1005E00090E0FC01EB57FD4F24918F589D4FFC018B
:1005F00084918823D1F090E0880F991FFC01E15C81
:10060000FD4FA591B491FC01E959FD4FC591D491DD
:1006100061110EC09FB7F8948C91E22FE0958E2364
:100620008C932881E223E8839FBFDF91CF910895C7
:100630008FB7F894EC91E22BEC938FBFF6CF8E300E
:1006400008F08E502091060190E4299F900111241A
:100650008770822B80937C0080917A0080648093E5
:100660007A0080917A0086FDFCCF8091780090918D
:10067000790008953FB7F8948091E8039091E903D9
:10068000A091EA03B091EB0326B5A89B05C02F3FCC
:1006900019F00196A11DB11D3FBFBA2FA92F982FA8
:1006A0008827BC01CD01620F711D811D911D42E0A3
:1006B000660F771F881F991F4A95D1F708958F926B
:1006C0009F92AF92BF92CF92DF92EF92FF926B0117
:1006D0007C010E943A034B015C01C114D104E10486
:1006E000F104B9F00E943A03681979098A099B0953
:1006F000683E73408105910580F321E0C21AD1085C
:10070000E108F10888EE880E83E0981EA11CB11C58
:10071000E4CFFF90EF90DF90CF90BF90AF909F908D
:100720008F9008958F929F92AF92BF92CF92DF9257
:10073000EF92FF920F931F93CF93DF938AE0A82E3F
:10074000B12CD0E0C0E0EE24EA9493E0F92E8824A6
:100750008A9423E0922ED12CC12C10E000E08FE08F
:100760000E941F030817190790F1C816D90608F44C
:100770006C018815990568F18E159F0508F47C01B8
:10078000C80FD91F65E070E080E090E00E945F0331
:1007900081E0A81AB10819F70C0D1D1DCE01801BB0
:1007A000910B8E199F098819990966E070E00E94E3
:1007B0009234CB01DF91CF911F910F91FF90EF9079
:1007C000DF90CF90BF90AF909F908F9008958C0155
:1007D000D0CF4C01D5CF2FB7F8946091E40370913E
:1007E000E5038091E6039091E7032FBF0895DC01B4
:1007F00080E0615090F09D919827E92FEF70F0E034
:10080000E15EFD4F2491E92FE295EF70F0E0E15DAC
:10081000FD4FE491822F8E27ECCF0895DC012C91BF
:100820001196ED91FC91F8948181822B81839281C4
:10083000322F30959323928387E090E00197F1F770
:1008400081818323818383E290E00197F1F7908196
:100850007894EFECF0E03197F1F7922381E009F41E
:1008600080E00895FC0190810180F281E02D292F24
:10087000209560FF14C0F894828182238283818155
:10088000892B8183A3E2B0E01197F1F78281982B45
:100890009283789487ED90E00197F1F70895F894AA
:1008A0008281822382838181892B8183AFEFB0E0B3
:1008B0001197F1F78281982B928378948FE090E0E2
:1008C000EBCFDF92EF92FF920F931F93CF93DF93C3
:1008D000EC01D62EE42E08E010E0FF24F39461E052
:1008E0008D2D8F2109F460E0CE010E943204FF0CAF
:1008F00001501109A1F7E11010C0F894E981FA81C3
:1009000091818881809589238183E981FA8192810F
:1009100088818095892382837894DF91CF911F917C
:100920000F91FF90EF90DF900895EF92FF920F9359
:100930001F93CF93DF938C017B0140E065E50E941C
:100940006104E70188E0E80EF11C699140E0C8010C
:100950000E946104CE15DF05C1F7DF91CF911F9191
:100960000F91FF90EF900895FC0190810180F2813A
:10097000E02DF8948181292F20958223818378941A
:100980003DE743E050E0315029F1DA011197F1F7EA
:1009900080818923C1F3F8948281822382838181BB
:1009A000892B81837894ABE7B7E01197F1F7F8943E
:1009B000818182238183A3E1B1E01197F1F78081E6
:1009C000982381E009F080E07894E3E6F6E031973F
:1009D000F1F7089580E008958F929F92AF92BF92B1
:1009E000CF92DF92EF92FF92CF93DF93EC018E8153
:1009F0009F810E94B40440E06CEC8E819F810E9434
:100A00006104488164E48E819F810E9461048A812F
:100A1000882371F1E981E9508EEEC82E82E0D82E4C
:100A2000E33038F4F0E0EE0FFF1FE35EFE4FC080CE
:100A3000D1808B81882339F18881811124C00E9463
:100A4000EB034B015C010D2C000CEE08FF088E81BE
:100A50009F810E940E04813059F00E94EB036C19B3
:100A60007D098E099F09681579058A059B0578F32C
:100A7000DF91CF91FF90EF90DF90CF90BF90AF903C
:100A80009F908F900895B601DD0C880B990BDF9134
:100A9000CF91FF90EF90DF90CF90BF90AF909F905D
:100AA0008F900C945F036F927F928F929F92AF9280
:100AB000BF92CF92DF92EF92FF920F931F93CF934B
:100AC000DF93EC017B018A018E819F810E94B40437
:100AD000811102C090E037C0B7018E819F810E94D2
:100AE000950440E06EEB8E819F810E946104780145
:100AF000680189E0C80ED11CAE80BF8088E0882ED6
:100B0000912C712C66246394C5010E940E048111FE
:100B10007628660CE1E08E1A9108B1F7F701719220
:100B20007F01EC15FD0541F78E819F810E94B40481
:100B3000813081F668E0C8010E94F70391E0F80176
:100B400020852813C7CF892FDF91CF911F910F9157
:100B5000FF90EF90DF90CF90BF90AF909F908F90DD
:100B60007F906F900895CF93DF93CDB7DEB729972D
:100B70000FB6F894DEBF0FBECDBFAE014F5F5F4F23
:100B80000E945305882331F08D818F33A9F020F422
:100B90008F31A1F080E007C08F3521F08F37D1F77A
:100BA0008CE001C08BE029960FB6F894DEBF0FBE33
:100BB000CDBFDF91CF9108958AE0F5CF89E0F3CFE3
:100BC0001F93CF93DF93EC01162F60E0812F0E94DB
:100BD000EE02612F70E0FB01EB57FD4FE491E883DB
:100BE000FB01EF58FD4FE491F0E0EE0FFF1FE35AD9
:100BF000FD4F859194919A8389831B861D861C865F
:100C00001A86198618861F821E821D821C821B82EC
:100C1000DF91CF911F9108952091FE033091FF0342
:100C20002817390771F49091FC038091FD03981700
:100C300041F0E091FC03F0E0ED55FC4F808190E045
:100C400008958FEF9FEF08950895EF92FF920F930D
:100C50001F93CF93DF93DC015C96ED90FC905D9742
:100C6000E114F10479F481E090E013969C938E9363
:100C7000129790E080E0DF91CF911F910F91FF904C
:100C8000EF9008955196ED91FC91529750968C916A
:100C90005097982F90950FB75E962C915E97122FD4
:100CA000127021FD6095F8942081112319F1282BF1
:100CB0002083E7012197F1F728E0462F50E03081AB
:100CC00060FF1AC0382B3083E7012197F1F7BA0192
:100CD00075956795215089F7112381F080818923CB
:100CE00080830FBF5C968D919C910197F1F781E015
:100CF00090E0C1CF2923DCCF3923E5CF9081892B28
:100D0000EFCF2091FE033091FF032817390771F4CC
:100D10008091FD032091FC0390E0805C9F4F821B3B
:100D2000910960E470E00E94A634089590E080E0AC
:100D300008952091FE033091FF0328173907B9F475
:100D40009091FC038091FD03981789F0E091FC03DA
:100D5000F0E0ED55FC4F80812091FC0330E02F5FE7
:100D60003F4F2F7333272093FC0390E008958FEFBC
:100D70009FEF08950F931F930E94EB036093FC0570
:100D80007093FD058093FE059093FF0584EF95E039
:100D90000E94990697FF1DC00E94EB030091FC057D
:100DA0001091FD052091FE053091FF05601B710B30
:100DB000820B930B0091F8051091F9052091FA052B
:100DC0003091FB056017710782079307F8F28FEFE8
:100DD0009FEF1F910F910895E091FE03F091FF03A3
:100DE000E817F90769F4A389B4899C9185898095EE
:100DF00089238C931092FF031092FE0381E00895E3
:100E000080E0089510920F0610920E0610920D06C3
:100E100010920C0610920B0610920A068DE991E0D2
:100E2000909311068093100690910006963108F079
:100E300046C02DEB30E030930B0620930A062BE9D9
:100E400031E030930D0620930C062CE231E0309314
:100E50000F0620930E062091680084E0983048F039
:100E600031E09E3008F430E081E001C0880F3A950F
:100E7000EAF7822B809368002DE630E0983050F03E
:100E80002BE630E09E3030F02CE630E0963110F06A
:100E900030E020E03093080620930706292F30E049
:100EA0009830C0F581E001C0880F9A95EAF78093E9
:100EB000090680911006909111060197F1F7809133
:100EC0000E0690910F06892B21F18091FE039091DF
:100ED000FF0325E0843F9207E1F0009711F00E94A4
:100EE000EC06809112068E7F809312061092FD030D
:100EF0001092FC0384EF95E09093FF038093FE0330
:100F0000E0910706F0910806808190910906892BEF
:100F1000808308959E3040F42850310981E001C05B
:100F2000880F2A95EAF7C3CF2E503109F7CF2091C9
:100F30008003260F3327331F21323105ECF4209133
:100F40004804FC0190E080E0243069F082E00895DC
:100F5000A09180032191AC01405A5C4FA40FB52FA2
:100F6000B11D2C930196861798F380918003680F2A
:100F70006093800380E0089581E008951092480412
:100F800081E0809347041092220461E082E10E9494
:100F9000A20261E083E10E94A202E9EBF0E080811D
:100FA0008E7F808380818D7F808388E48093B800EA
:100FB00085E48093BC00089510920104109200040F
:100FC00010924F04109271040E94BE0789E791E0CD
:100FD0009093FB038093FA038AE791E09093F903DF
:100FE0008093F8030895CF93DF9391E090935F038C
:100FF0008823B9F0C091B800D091BA008091BC00AC
:101000008A7B8093BC0060E082E10E94A20260E0E3
:1010100083E10E94A2020E94BE07D093BA00C0934F
:10102000B800DF91CF910895CF92DF92EF92FF92B7
:101030000F931F93CF93DF93D091710481E0D1324E
:1010400008F09CC0C09170040E943A036B017C01BF
:101050008091480481116CC082E08093480481E053
:10106000809347048FEF8093460410924504D093F9
:101070004404A0E5B4E0E4E2F4E080E0D8138DC0DD
:101080001092230480912304CC0FC82BC093230417
:1010900080912204813009F084C0109222040E94C1
:1010A0003A036B017C01809123048093BB00809103
:1010B0004A0490914B04A0914C04B0914D04892BAB
:1010C0008A2B8B2BA1F00E943A0300914A041091C5
:1010D0004B0420914C0430914D046C197D098E090C
:1010E0009F09061717072807390708F442C080919F
:1010F000BC0083FDD8CF85EC8093BC000E943A03EE
:101100006B017C0180914804823009F44CC08091CD
:1011100046048F3F09F469C080914604803209F487
:1011200066C080914604803309F463C084E026C021
:1011300080914A0490914B04A0914C04B0914D04CD
:10114000892B8A2B8B2B09F483CF0E943A030091C1
:101150004A0410914B0420914C0430914D046C19B9
:101160007D098E099F09061717072807390708F018
:101170006FCF809149040E94F30785E010924F04DD
:101180001092710410924E04DF91CF911F910F9134
:10119000FF90EF90DF90CF9008959D9191938F5F96
:1011A0006DCF85EEA9CF80914A0490914B04A09118
:1011B0004C04B0914D04892B8A2B8B2B09F4A2CFC0
:1011C0000E943A0300914A0410914B0420914C0470
:1011D00030914D046C197D098E099F090617170778
:1011E0002807390708F08ECFC4CF80E0C7CF82E050
:1011F000C5CF83E0C3CFCF92DF92EF92FF920F93E0
:101200001F93CF93DF93D82FC62F613208F098C079
:101210000E943A036B017C018091480481116BC0EC
:1012200081E080934804809347049FEF90934604A5
:10123000109245049C0F9093440480932304809162
:101240002304DD0FD82BD093230480912204813016
:1012500009F078C0109222040E943A036B017C01CD
:10126000809123048093BB0080914A0490914B04A9
:10127000A0914C04B0914D04892B8A2B8B2BA1F0AB
:101280000E943A0300914A0410914B0420914C04AF
:1012900030914D046C197D098E099F0906171707B7
:1012A0002807390708F448C08091BC0083FDD8CFD7
:1012B00085EC8093BC000E943A036B017C01809115
:1012C0004804813009F440C0809145048C1710F423
:1012D000C0914504E4E2F4E0A2E0B4E080E08C13C5
:1012E00055C08C2FDF91CF911F910F91FF90EF9000
:1012F000DF90CF90089580914A0490914B04A09183
:101300004C04B0914D04892B8A2B8B2B09F484CF8C
:101310000E943A0300914A0410914B0420914C041E
:1013200030914D046C197D098E099F090617170726
:101330002807390708F070CF809149040E94F3070D
:10134000C0E0CFCF85EEB5CF80914A0490914B0499
:10135000A0914C04B0914D04892B8A2B8B2B09F45E
:10136000AECF0E943A0300914A0410914B042091A1
:101370004C0430914D046C197D098E099F090617A4
:1013800017072807390708F09ACFD6CF91919D9378
:101390008F5FA5CFE091010480910004E81730F43D
:1013A000F0E0EE5FFB4F808190E008958FEF9FEFBC
:1013B000089590910104809100042FEF3FEF98175A
:1013C00048F4E92FF0E0EE5FFB4F208130E09F5FB3
:1013D00090930104C9010895809100049091010443
:1013E000891B990B0895CF92DF92EF92FF920F9392
:1013F0001F93CF93DF937C01CB018A0120914E0490
:10140000222389F0EB016B01C40ED51ECC15DD053E
:1014100069F06991D701ED91FC910190F081E02D87
:10142000C7010995F3CF642F0E949707C801DF9188
:10143000CF911F910F91FF90EF90DF90CF90089583
:10144000CF93DF931F92CDB7DEB7698320914E040F
:101450002223F9F020917104203258F021E030E08D
:10146000FC013383228390E080E00F90DF91CF91E5
:10147000089580914F04E82FF0E0E05BFB4F9981E5
:1014800090838F5F80934F048093710481E090E09C
:10149000ECCF61E0CE0101960E949707F7CF90E074
:1014A00080E0089584EF95E00E94EC060C9402071A
:1014B0002F923F924F925F926F927F928F929F9264
:1014C000AF92BF92CF92DF92EF92FF920F931F9352
:1014D000CF93DF93CDB7DEB72D970FB6F894DEBF6D
:1014E0000FBECDBF1C010E94520A64E670E080E08E
:1014F00090E00E945F036AE070E080E090E00E946C
:101500005F03C101880F991F9D878C87D12CC12C47
:10151000F12CE12C412C512C320149E050E064E1E6
:1015200071E084EF95E00E947C0165E070E080E06E
:1015300090E00E945F0310E000E0812C912C5401A8
:1015400084EF95E00E948106892B39F4F4E08F1630
:101550009104A104B1040CF05FC0023011050CF03D
:101560005BC084EF95E00E948106892B99F084EF9F
:1015700095E00E949906E1E0F0E0EC0FFD1FE00F1E
:10158000F11F80836AE070E080E090E00E945F03DA
:101590000F5F1F4F65E070E080E090E00E945F0306
:1015A0000230110509F070C089818F3F09F06CC0CD
:1015B0008A81863809F068C0FE013396FB87EA8786
:1015C00084EF95E00E948106892B39F4F4E08F16B0
:1015D0009104A104B1040CF050C00930110509F0C8
:1015E00059C08B8190E0982F88272C81820F911D04
:1015F000092E000CAA0BBB0B480E591E6A1E7B1E3F
:1016000040C0EC85FD85EC15FD0509F086CFE114A1
:10161000F10441F4710106C08FEFC81AD80AE21430
:10162000F3047CF3C301B2010E9403304B015C015F
:10163000B701FF0C880B990B0E9403309B01AC0192
:10164000C501B4010E94F7312D960FB6F894DEBFA4
:101650000FBECDBFDF91CF911F910F91FF90EF9003
:10166000DF90CF90BF90AF909F908F907F906F90C2
:101670005F904F903F902F900895043011050CF02B
:10168000B0CFFFEFEF1AFF0A8FEF881A980AA80A67
:10169000B80A56CF84EF95E00E949906EA85FB854B
:1016A0008193FB87EA870F5F1F4F8ACF8F929F92AC
:1016B000AF92BF92CF92DF92EF92FF92CF93DF93E0
:1016C000C6ECD5E0988121E020934E0490937004FD
:1016D00010924F0410927104682F8FE095E00E94E1
:1016E000200A0E94140863E088810E94FB0810927F
:1016F0000104809300048FE095E00E94D909092E2F
:10170000000CAA0BBB0B8824982EA92EBA2E8FE0B2
:1017100095E00E94D909092E000CAA0BBB0B6C01A5
:101720007D01C828D928EA28FB28FE2CED2CDC2CCA
:10173000CC248FE095E00E94D909BC01990F880B59
:10174000990B6C297D298E299F29DF91CF91FF90DC
:10175000EF90DF90CF90BF90AF909F908F900895C3
:101760008F929F92AF92BF92CF92DF92EF92FF92B1
:101770000F931F932091CF052F3F19F48AEF0E94FA
:10178000560B0091D3051091D40530E020E0C72E10
:10179000D82EE92EFF24E7FCFA94C01AD10AE20AF7
:1017A000F30A57E095958795779567955A95D1F700
:1017B000000F111F221F331F4B015C01801A910A79
:1017C000A20AB30AA5019401A091D505B091D6054E
:1017D0000E94E2344B015C01FBE0B594A79497941E
:1017E0008794FA95D1F7A7019601C701B6010E9427
:1017F00082349B01AC01ACE0559547953795279510
:10180000AA95D1F7A091D705B091D8050E94E234EE
:101810009B01AC01BEE05595479537952795BA9544
:10182000D1F7280D391D4A1D5B1D2093CB05309340
:10183000CC054093CD055093CE05A5E0B0E00E94C5
:10184000393160587F4F8F4F9F4F672F782F892FE7
:10185000992787FD9A950E94033020E030E048ECFC
:1018600052E40E94F7311F910F91FF90EF90DF90AB
:10187000CF90BF90AF909F908F9008952F923F92FE
:101880004F925F926F927F928F929F92AF92BF9290
:10189000CF92DF92EF92FF920F931F93CF93DF933C
:1018A000CDB7DEB76B970FB6F894DEBF0FBECDBFD6
:1018B0000E94B00B8091CF058F3F39F487EF0E94D3
:1018C000560B6E8B7F8B888F998F8091CB05909173
:1018D000CC05A091CD05B091CE056C017D01FF0C2A
:1018E000CC08DC2C76019C01AD016C2D7C2D8C2D5F
:1018F0009C2D345F414051096109710981099109A9
:1019000029873A874B87652E762E872E982E9B8FB8
:101910005901C42ED52EE62EF72E082F192F0E941E
:10192000EA34322E232E488B598B6A8B7B8B8C8B1F
:101930009D8B3091DC052091DB05932F990F990B3E
:10194000492F592F692F792F892F0E94EA340CE0F3
:101950000E94E23529833C874A8F5D876E877F87A7
:10196000582E492E3091DE052091DD05932F990FD9
:10197000990BA32CB22CC888D988EA88FB880C89DB
:101980001D89492F592F692F792F892F0E94EA34F9
:1019900008E00E94FB35A980BC84CA8CDD84EE84FB
:1019A000FF84052D142D0E94183670588F4F9F4FBD
:1019B000E091D905F091DA055F01D12CC12CE12C21
:1019C000F12C8701E983BA82CB82DC82ED82FE8230
:1019D0000F831887C12CD12CE12CF12C00E010E0F2
:1019E0000E94EA3401E20E94FB352A8F532E49837C
:1019F0005C876D877E878F87492EA0E00E942A36FC
:101A000009F436C13091E4052091E305932F990F35
:101A1000990BA32CB22CC888D988EA88FB880C893A
:101A20001D89492F592F692F792F892F0E94EA3458
:101A30001901488B598B6A8B7B8B8C8B9D8B3091DA
:101A4000E2052091E105932F990F990BA984BA849F
:101A5000CB84D62CE72CF82C092D1B8D492F592F20
:101A6000692F792F892F0E94EA3401E10E94E23523
:101A70005101C888D988EA88FB880C891D890E9491
:101A8000183659016A017B01382E192F4E895F895A
:101A9000688D798D84E075956795579547958A95FA
:101AA000D1F780E090E0A0E1B0E0841B950BA60B9D
:101AB000B70B3C014D01990C6608762C43019C0143
:101AC000AD01662D762D862D962D0FE10E94E23513
:101AD000722E832E942E5987B62FA72FF82FE92F19
:101AE0003091E0052091DF05932F990F990B492F35
:101AF000592F692F792F892F03E20E94E235032D98
:101B00000E94183659016A017B018C01272D382D5E
:101B1000492D59856B2F7A2F8F2F9E2F0E942136AA
:101B2000E5E3AE2EFCE0BF2EC12CD12CE12CF12C34
:101B300000E010E00E94EA34AA8CB52CC980DC8455
:101B4000ED84FE840F85142D0E9444352F873E8737
:101B500049875A876B8779838C879D870DE00E9420
:101B6000FB35922E832E742E652E562E472E382E40
:101B7000292E3091EA052091E905932F990F990BB1
:101B8000A92CB82CC72CD62CE52CF42C032D122D07
:101B9000492F592F692F792F892F0E94EA340E94EB
:101BA000EA3409E10E94FB35AF84BE84C984DA843B
:101BB000EB84F9800C851D850E94183619012A01D5
:101BC0003B014C013091E8052091E705932F990FD7
:101BD000990B492F592F692F792F892F0E94EA34A9
:101BE00003E10E94FB3559016A017B018C019101DF
:101BF000A201B301C4010E94183608E00E94FB351F
:101C000059016A017B01E82F192F3091E6052091D7
:101C1000E505932F990F990B492F592F692F792F8C
:101C2000892F04E00E94E2350E2F0E9418360E9490
:101C30009F3220E030E040E85BE30E9462306B9628
:101C40000FB6F894DEBF0FBECDBFDF91CF911F91CD
:101C50000F91FF90EF90DF90CF90BF90AF909F904B
:101C60008F907F906F905F904F903F902F9008954E
:101C700060E070E0CB01E3CFBF92CF92DF92EF92B2
:101C8000FF920F931F93CF93DF93EC01B62EC72ED5
:101C90008D85811105C0CE010E94B40481110EC052
:101CA0001B861D861C8680E0DF91CF911F910F91CE
:101CB000FF90EF90DF90CF90BF90089540E060EFED
:101CC000CE010E94610401E0E12CD12C11E0CE0193
:101CD0000E940E04F82ECE010E940E0491E0F9122B
:101CE00018C0813099F51134D8F2DB86D11002C0CA
:101CF00081E08D878B81882399F22396EB2DFC2D33
:101D0000CF01089629912193E817F907D9F781E0C7
:101D1000CBCFEE2DF0E0F8120FC08B851817A0F492
:101D2000DE01AE0FBF1F13968C91802379F4F12C46
:101D3000193008F41C87D12EEC0FFD1F8381902FE2
:101D40009095892383830AC08113F1CFFE01EE0DA4
:101D5000F11D8381802B8383FF24F3946F2DCE01AB
:101D60000E9432041F5F000F11F4E39401E087E04A
:101D70008E1508F0ACCFB7CFDF92EF92FF920F93A2
:101D80001F93CF93DF937C018B01D42EDC01169639
:101D9000ED91FC91138615861486128611861086A5
:101DA00017821682158214821382C0E0B801F701EF
:101DB000868197810E943C0ED82F882329F0DC165B
:101DC00029F0CF5FDC1690F7D0E009C067E0C801CA
:101DD0000E94F703D80117969C918913F2CF8D2F9B
:101DE000DF91CF911F910F91FF90EF90DF900895B9
:101DF0000F931F93CF93DF93CDB7DEB761970FB6E5
:101E0000F894DEBF0FBECDBF8C01462FBE01665FCA
:101E10007F4F0E94BC0E81110FC060E070E08EEF1A
:101E200092EC61960FB6F894DEBF0FBECDBFDF9186
:101E3000CF911F910F910895AE014F5F5F4FBE018B
:101E4000665F7F4FC8010E945305882331F36A8182
:101E500070E0762F6627770F770F770F298148E09C
:101E6000249F90011124262B372B8A858031D1F4B1
:101E7000688570E08F81AB01481B5109CA019695B6
:101E8000982F8827979587950E94A634CB01409775
:101E9000B90153E0660F771F5A95E1F760789C010E
:101EA000260F371F213854EE35070CF4B6CFB90191
:101EB000330F880B990B0E94033020E030E040E0A4
:101EC0005CE30E946230ADCFEF92FF920F931F93BD
:101ED000CF93DF93CDB7DEB728970FB6F894DEBF68
:101EE0000FBECDBF8C01DC011696ED91FC911797CA
:101EF000138615861486128611861086178216821E
:101F000015821482138214961C92149715961C92B3
:101F1000EE24E394BE016F5F7F4FF80186819781C5
:101F20000E943C0E882309F46FC067E0CE01019641
:101F30000E94F70398858913EDCFD8018C91811108
:101F400025C016968D919C910E94B404BE016F5FCE
:101F50007F4FF801868197810E94950440E064EBF1
:101F6000D80116968D919C910E946104F80186819A
:101F700097810E940E04F82ED80116968D919C919F
:101F80000E94B404F11002C0F801E082D801119659
:101F9000FC9089818031A1F1BE016F5F7F4FC80144
:101FA0000E94B3058F15D0F4F8018181D8011196F4
:101FB0008C93119714968C9114978F5F14968C9331
:101FC0008981883231F0B0F4803119F0823209F021
:101FD000A1CFF80185818F5F85839CCF8981803176
:101FE00011F48CE0E3CFBE016F5F7F4FC8010E9408
:101FF000B305DCCF8B3369F3823409F08BCFE9CFA3
:10200000FCE0FF1588F2EDCF28960FB6F894DEBFFE
:102010000FBECDBFDF91CF911F910F91FF90EF9039
:1020200008959F92AF92BF92CF92DF92EF92FF926C
:102030000F931F93CF93DF93CDB7DEB761970FB6A2
:10204000F894DEBF0FBECDBF8C018CE0F801818318
:10205000D12CC12C2FE5E22E3FE7B32E4FE1A42E69
:102060005FE3952EF80184818C151D0409F00CF4B2
:10207000A3C04C2DBE01665F7F4FC8010E94BC0EFD
:10208000F801F180FCE0FF1550F59CE0F92E8A85FF
:10209000803159F1BE01665F7F4FC8010E94B305D0
:1020A000F81609F481C0AE014F5F5F4FBE01665F55
:1020B0007F4FC8010E945305882309F475C08A85A3
:1020C000803109F471C0EBE0FE1609F471C0FCE048
:1020D000FF1669F08AE0F8126DC09D8209C089E0A0
:1020E000F816A8F689E0F82ED2CF8CE0D9CFBD82C1
:1020F000F801868197810E94B404BE01665F7F4F1C
:10210000F801868197810E94950440E06EE4F80111
:10211000868197810E94610440E06B81F80186818D
:1021200097810E94610440E06C81F801868197816B
:102130000E9461048A85803139F040E06D81F801A8
:10214000868197810E946104F801868197810E94AF
:10215000B404BE01665F7F4FF801868197810E94BB
:102160009504F801408168E4868197810E946104AA
:1021700064E170E080E090E00E945F03F8018081FC
:10218000882331F06AE070E080E090E00E945F0315
:10219000F801868197810E94B404F80181818F152E
:1021A00008F48F2DF8018183FFEFCF1ADF0A5ACF91
:1021B000ED829ECFAD829CCF61960FB6F894DEBFC4
:1021C0000FBECDBFDF91CF911F910F91FF90EF9088
:1021D000DF90CF90BF90AF909F900895CF93909154
:1021E000CF059F3F41F5682F8091C60591E0909300
:1021F0004E048093700410924F04109271048FE08B
:1022000095E00E94200A0E94140862E08091C605B1
:102210000E94FB0810920104809300048FE095E077
:102220000E94D909C82F8FE095E00E94D90920E0CB
:102230003C2F282B392B922F832FCF9108950F936A
:102240001F93CF93DF93FC010481158101151105C4
:1022500039F4FB011082DF91CF911F910F91089506
:10226000415051094017510708F48A01EB01FC0164
:1022700060817181A801CE010E943E38C00FD11F3C
:102280001882E9CFCF93DF93C091BA05D091BB05F7
:10229000209761F08991882349F0082E000C990B52
:1022A0000E941838FE0131978083F4CFDF91CF91DF
:1022B000089585ED8093BC0080914A0490914B0471
:1022C000A0914C04B0914D040796A11DB11D23E0CF
:1022D000B695A795979587952A95D1F72091BC003B
:1022E00024FD03C010924804089540914A0450917F
:1022F0004B0460914C0470914D04452B462B472BA9
:1023000069F30097A105B10541F025E32A95F1F79E
:1023100000000197A109B109E1CF809149040C9413
:10232000F307FC0180819181009711F00C94E32B5D
:1023300060E070E0CB010895FB0144815581FC0110
:10234000248135812417350778F0808191810097A9
:1023500059F0FB01608171816115710529F00E94BE
:10236000303821E0892B09F020E0822F08950F9367
:102370001F93CF93DF938C01EB01FC01808191814E
:102380000097E1F06881798161157105A9F04281BA
:1023900053812C813D814217530770F00E942938E8
:1023A0008C819D81F801958384831D821C82DF913D
:1023B000CF911F910F9108950E94D2368881998103
:1023C000F801918380838A819B81938382838C81AE
:1023D0009D8195838483198218821B821A82E5CF9E
:1023E000CF93DF93EC0188819981009711F00E94CF
:1023F000D236198218821D821C821B821A82DF91BA
:10240000CF910895FC0180819181009711F00C9487
:10241000D23608950F931F93CF93DF93EC018881F9
:102420009981009759F02A813B812617370730F0B0
:1024300081E0DF91CF911F910F9108958B016F5F24
:102440007F4F0E945B37009759F0998388831B83E5
:102450000A832C813D81232B59F7FC011082E8CFA0
:1024600080E0E7CFEF92FF920F931F93CF93DF931C
:102470006115710541F480E0DF91CF911F910F91BB
:10248000FF90EF90089541155105B1F07B01EC01EB
:102490000C811D81040F151FB8010E940A128823A8
:1024A00051F3288139818C819D81B701820F931F5F
:1024B0000E9429381D830C8381E0DECFFC0144811A
:1024C00055816081718180EC95E00C9432120F93FC
:1024D0001F93CF93DF9300D0CDB7DEB78C01698314
:1024E0001A8241E050E0BE016F5F7F4F0E943212BE
:1024F000811103C0C8010E94F011C8010F900F9014
:10250000DF91CF911F910F910895CF93DF93EC014D
:10251000FB0101900020E9F73197AF01461B570BF3
:102520000E943212811103C0CE010E94F011CE012F
:10253000DF91CF910895CF93DF93EC01FB014481AC
:102540005581608171810E943212811103C0CE01D8
:102550000E94F011CE01DF91CF910895EF92FF928A
:102560000F931F93CF93DF93EC017B018A01BA0194
:102570000E940A1281110BC0CE010E94F011CE01FF
:10258000DF91CF911F910F91FF90EF9008951D83E0
:102590000C83B701888199810E942938F0CFFB0113
:1025A00001900020E9F73197AF01461B570B0C94BF
:1025B000AE120F931F93CF93DF93CDB7DEB7629721
:1025C0000FB6F894DEBF0FBECDBF8C01CB01F80172
:1025D0001182108213821282158214824AE0BE0197
:1025E0006F5F7F4F0E940A2CBE016F5F7F4FC80153
:1025F0000E94CF1262960FB6F894DEBF0FBECDBF19
:10260000DF91CF911F910F910895CF93DF93EC014C
:10261000FB018617970749F060817181611571058B
:1026200041F0448155810E94AE12CE01DF91CF91DD
:1026300008950E94F011F9CFFC01118210821382DB
:102640001282158214820C940513FC0111821082EF
:102650001382128215821482FB0101900020E9F797
:102660003197AF01461B570B0C94AE12AF92BF923D
:10267000CF92DF92EF92FF920F931F93CF93DF934E
:102680006C015B017A0189012417350720F48F2D35
:102690007901042F182F6BE571E0C6010E94251304
:1026A000D5011496CD91DC91EC16FD06E0F40C17E3
:1026B0001D0708F4E801D501ED91FC911197EC0F8D
:1026C000FD1F108110826D917C916E0D7F1DC601E2
:1026D00061157105A1F00E94CF12F50180819181F1
:1026E000C80FD91F1883C601DF91CF911F910F9199
:1026F000FF90EF90DF90CF90BF90AF9008950E9431
:10270000F011EBCFCF93DF93EC01FB0124813581F6
:102710000E943613CE01DF91CF9108950F931F933E
:10272000CF93DF93CDB7DEB72C970FB6F894DEBF0B
:102730000FBECDBFFC01248135811216130664F44F
:102740008C01253131059CF40E94A90164E170E0FF
:1027500080E090E00E945F032C960FB6F894DEBFF5
:102760000FBECDBFDF91CF911F910F9108952FE044
:1027700030E050E040E0BC01CE0107960E943613E5
:102780004B855C856F81788582E794E00E947C01AF
:1027900069E170E080E090E00E945F034FE050E06C
:1027A000B801CE0101960E948213BE016F5F7F4F78
:1027B000CE0107960E94B711CE0101960E94021227
:1027C000CE0107960E94A90164E170E080E090E0EC
:1027D0000E945F036BE571E0CE0107960E94CF1265
:1027E000CE0107960E940212B7CFEF92FF920F938D
:1027F0001F93CF93DF93CDB7DEB7A1970FB6F894B1
:10280000DEBF0FBECDBF7C01CB01BA01F701118243
:102810001082138212821582148242E0420F8E01CE
:102820000F5F1F4F0E94C12B009789F0BC01C701A9
:102830000E94CF12A1960FB6F894DEBF0FBECDBF97
:10284000DF91CF911F910F91FF90EF900895C701F5
:102850000E94F011EFCFFF920F931F93CF93DF935E
:10286000EC01F62E08811981C8010E942331F81667
:1028700021F06F2DC8010E942B31CE01DF91CF9145
:102880001F910F91FF900895EF92FF920F931F9366
:10289000CF93DF9300D0CDB7DEB70BE115E08B51BE
:1028A00095407C01C701800F911F9A838983F801AD
:1028B00061918F01CE0101960E942B14F5E009363B
:1028C0001F0781F78BE195E00F900F90DF91CF917B
:1028D0001F910F91FF90EF900895EF92FF920F9349
:1028E0001F93CF93DF9300D0CDB7DEB70FE615E08F
:1028F0008F5695407C01C701800F911F9A83898371
:10290000F80161918F01CE0101960E942B14F5E030
:1029100006391F0781F78FE695E00F900F90DF9142
:10292000CF911F910F91FF90EF9008952F923F92BA
:102930004F925F926F927F928F929F92AF92BF92CF
:10294000CF92DF92EF92FF920F931F93CF93DF937B
:10295000CDB7DEB7E6970FB6F894DEBF0FBECDBF9A
:102960006EEA75E08AEB95E00E9405130E94421121
:102970006CE571E0CE0101960E942513BE016F5FE8
:102980007F4F8AEB95E00E949C11182FCE01019693
:102990000E940212112329F0F0E0E0E0099581E0A5
:1029A00092C060E671E0CE0101960E942513BE013F
:1029B0006F5F7F4F8AEB95E00E949C11182FCE012C
:1029C00001960E940212112351F164E671E0CE01DA
:1029D00001960E94251366E975E0CE0101960E94DA
:1029E0009B12BC0180EC95E00E940513CE0101967C
:1029F0000E94021260EC75E0CE0101960E941C1349
:102A0000CE0101960E948E13CE0101960E94021201
:102A10006BE571E080EC95E00E94CF12C0CF6EE6CE
:102A200071E0CE0101960E942513BE016F5F7F4FBA
:102A30008AEB95E00E949C11182FCE0101960E940E
:102A40000212112359F062E771E080EC95E00E94D8
:102A5000CF128CE995E00E945E12CCCF60E871E065
:102A6000CE0101960E942513BE016F5F7F4F8AEB56
:102A700095E00E949C11182FCE0101960E9402122F
:102A80001123D1F127E030E046E050E06EEA75E036
:102A9000CE0101960E943613BE016F5F7F4F88EA18
:102AA00095E00E94B711CE0101960E94021288EAB9
:102AB00095E00E949111672B19F41092EE036FCFED
:102AC00081E08093EE03E6960FB6F894DEBF0FBE6A
:102AD000CDBFDF91CF911F910F91FF90EF90DF90CD
:102AE000CF90BF90AF909F908F907F906F905F90AE
:102AF0004F903F902F90089567E871E0CE010196C6
:102B00000E942513BE016F5F7F4F8AEB95E00E9404
:102B10009C11182FCE0101960E940212112309F474
:102B2000B8C080915D0390915E03181619060CF0F1
:102B300036CF88EC90E0909305018093040182E702
:102B400094E00E9482021BA21CA21DA21EA2CC2401
:102B5000C394D12CA0EC2A2EA3E03A2E5E01F3E21E
:102B6000AF0EB11C2E0127E2420E511CBDE56B2EAB
:102B7000B3E07B2E80915D0390915E038C159D05E3
:102B80000CF40DCF8091040190910501813C93409C
:102B900024F030920501209204010091040110916B
:102BA0000501750148018A189B08C4018E0D9F1DFF
:102BB0000E942331F70181937F01E415F505A9F700
:102BC000C80104969093050180930401E9E3EE2E79
:102BD000E3E0FE2E05531340C8018E0D9F1D0E9499
:102BE0002331F70181937F016E167F06A9F74BA170
:102BF0005CA16DA17EA123E0CE0145960E94F51354
:102C0000BE016B5E7F4FCE0101960E941C136BE8E4
:102C100071E0CE0101960E948512BC0180EC95E026
:102C20000E940513CE0101960E940212CE01459624
:102C30000E94021269E373E0CE0101960E942513FF
:102C4000CE0101960E945E12CE0101960E940212F0
:102C500060EC75E0CE0101960E941C13CE01019636
:102C60000E948E13CE0101960E94021280910401EF
:102C7000909105018496909305018093040164E18D
:102C800070E080E090E00E945F03FFEFCF1ADF0A60
:102C900071CF6EE871E0CE0101960E942513BE014E
:102CA0006F5F7F4F8AEB95E00E949C11182FCE0139
:102CB00001960E9402121123F1F126E030E045E076
:102CC00050E06EEA75E0CE0101960E943613BE0117
:102CD0006F5F7F4F88EA95E00E94B711CE010196A1
:102CE0000E94021288EA95E00E949111672B19F464
:102CF0001092380354CE81E08093380388EC90E042
:102D0000909305018093040110925E0310925D037D
:102D10001092340310923503109236031092370349
:102D20000E94EB036093300370933103809332036E
:102D30009093330334CE64E971E0CE0101960E9492
:102D40002513BE016F5F7F4F8AEB95E00E949C11B7
:102D5000182FCE0101960E940212112309F46DC0B2
:102D60008091B2059091B305079708F418CE46E01C
:102D700050E06EEA75E0CE0101960E948213BE011A
:102D80006F5F7F4F88EA95E00E94B711CE010196F0
:102D90000E9402120E9465266B017C01C0920A010A
:102DA000D0920B01E0920C01F0920D016BE971E001
:102DB00080EC95E00E94CF1222E0B701A601CE017F
:102DC00045960E94F513BE016B5E7F4FCE010196C2
:102DD0000E941C1364EC72E0CE0101960E948512E1
:102DE0000E945E12CE0101960E940212CE0145960B
:102DF0000E94021260EC75E0CE0101960E941C1345
:102E0000CE0101960E948E13CE0101960E940212FD
:102E10000E94EB0328EE33E040E050E00E94BA3419
:102E2000CA01B9010E9401306093F3037093F40367
:102E30008093F5039093F603B2CD66EA71E0CE017C
:102E400001960E942513BE016F5F7F4F8AEB95E0CC
:102E50000E949C11182FCE0101960E94021211238C
:102E600009F459C08091B2059091B305079708F411
:102E700096CD46E050E06EEA75E0CE0101960E94E4
:102E80008213BE016F5F7F4F88EA95E00E94B71101
:102E9000CE0101960E9402120E9465266B017C0100
:102EA000C0920001D0920101E0920201F092030170
:102EB0006DEA71E080EC95E00E94CF1221E0B7014D
:102EC000A601CE0145960E94F513BE016B5E7F4FB1
:102ED000CE0101960E941C1364EC72E0CE010196B3
:102EE0000E9485120E945E12CE0101960E9402127B
:102EF000CE0145960E94021260EC75E0CE0101966B
:102F00000E941C13CE0101960E948E13CE010196E1
:102F10000E94021244CD68EB71E0CE0101960E943E
:102F20002513BE016F5F7F4F8AEB95E00E949C11D5
:102F3000182FCE0101960E9402121123D9F143E00D
:102F400050E06EEA75E0CE0101960E948213BE0148
:102F50006F5F7F4F88EA95E00E94B711CE0101961E
:102F60000E94021268EA75E0CE0101960E941C13CD
:102F700060E0CE0101960E946712BC018CE995E0E9
:102F80000E940513CE0101960E9402124091A005F5
:102F90005091A1054115510531F06DE175E08CE9C5
:102FA00095E00E941F1180910801909109010E94F3
:102FB0004414F5CC6FEB71E0CE0101960E9425130D
:102FC000BE016F5F7F4F8AEB95E00E949C11182F26
:102FD000CE0101960E940212112309F478C080915B
:102FE000B2059091B305409708F027C442E050E045
:102FF0006EEA75E0CE0101960E948213BE016F5FFA
:103000007F4F88EA95E00E94B711CE0101960E9499
:1030100002120E94652620E030E048EC52E40E9453
:1030200062300E946932609327057093280580936F
:10303000290590932A056CEB71E080EC95E00E94E5
:10304000CF126091270570912805809129059091F4
:103050002A058B019C0100591F452140310901348B
:103060001C492105310598F068EA75E0CE0101960A
:103070000E941C1362EC71E0CE0101960E94851241
:103080000E945E12CE0101960E94021288CC0E941C
:10309000033020E030E048EC52E40E94F731AB010D
:1030A000BC0122E0CE0101960E94F513CE010196EB
:1030B0000E945E12CE0101960E94021243E050E08F
:1030C0006FEC71E080EC95E00E9432126CCF63ED02
:1030D00071E0CE0101960E942513BE016F5F7F4F04
:1030E0008AEB95E00E949C11182FCE0101960E9458
:1030F00002121123F1F025E030E044E050E06EEAE6
:1031000075E0CE0101960E943613BE016F5F7F4FBE
:1031100088EA95E00E94B711CE0101960E94021242
:1031200088EA95E00E9491117093680560936705A5
:103130003ACF68ED71E0CE0101960E942513BE01E1
:103140006F5F7F4F8AEB95E00E949C11182FCE0194
:1031500001960E940212112309F45EC009E110E0F9
:10316000C12CD12C760180E10E941F03BC01990F74
:10317000880B990B0E9403309B01AC01C701B6017B
:103180000E948B316B017C016AE070E080E090E08E
:103190000E945F030150110931F720E030E040EA5E
:1031A00050E4C701B6010E94623020E030EC4FE7E6
:1031B00054E40E94F73120E030E048EC51E40E94F2
:1031C000F7316093430570934405809345059093D0
:1031D000460580910801909109010E9444146CED0C
:1031E00071E080EC95E00E94CF1240914305509130
:1031F0004405609145057091460522E0CE01459653
:103200000E94F513BE016B5E7F4FCE0101960E94B6
:103210001C1364EE71E062CE67EE71E0CE010196A0
:103220000E942513BE016F5F7F4F8AEB95E00E94DD
:103230009C11182FCE0101960E940212112309F44D
:103240004EC126E030E044E050E06EEA75E0CE0189
:1032500001960E943613BE016F5F7F4F88EA95E0AA
:103260000E94B711CE0101960E94021288EA95E0F1
:103270000E9491112B017B016E0185E1C80ED11CCA
:1032800067E772E0C6010E9425138091B205909114
:10329000B305298D3A8D5C01A21AB30A21153105B7
:1032A00069F1009759F18217930740F1A816B90602
:1032B00020F05C01E1E0AE1AB1088090AE0590907C
:1032C000AF052D893E893EAB2DABC4010FEF1FEF3B
:1032D00014012A0C3B1C2816390690F06DA97EA912
:1032E0000E944D38009761F09C0128193909A216F7
:1032F000B30608F4980101968901EDCF0FEF1FEF97
:10330000A8014F5F5F4F6EEA75E0CE0101960E9403
:103310008213BE016F5F7F4F88EA95E00E94B7116C
:10332000CE0101960E940212C6010E9402120E9462
:1033300065264B015C01120131E0231A31086FE070
:10334000C6010E94E005D886CF821D821E821982A6
:1033500089E08A8381E08B838C831C8A1B8ACE015F
:1033600001960E94640FCE0101960E94EC04CE01EA
:1033700001960E9411100E8110E00530110514F025
:1033800004E010E04BE54416510408F44DC077E426
:10339000C72E75E0D72E812C912C5401F12CE12CF5
:1033A0000E151F05B9F06E2DCE0101960E94F80E84
:1033B0009B01AC01F60121933193419351936F012D
:1033C000C501B4010E948B314B015C01FFEFEF1A84
:1033D000FF0AE6CFB7010F2C000C880B990B0E9457
:1033E00003309B01AC01C501B4010E94F7314B01D0
:1033F0005C010BE115E0D12CC12C0C5F1F4FEC14CC
:10340000FD0499F1F80120A531A542A553A5C501F8
:10341000B4010E948A31F80160A771A782A793A71F
:10342000FFEFCF1ADF0AE9CF1E141F04CCF50E15EB
:103430001F0524F4180121E0221A3108622DCE0163
:1034400001960E94F80E9B01AC018101000F111F33
:10345000000F111F095B1A4FC501B4010E948A3188
:10346000F801608371838283938380910801909136
:1034700009010E9444146BEE71E080EC95E00E941B
:10348000CF1244E050E06EEA75E0CE0101960E9452
:103490008213CE0101960E945E12CE0101962ACDC2
:1034A000E114F10411F727E4C22E25E0D22E0E1507
:1034B0001F05D9F26E2DCE0101960E94F80E9B01D8
:1034C000AC01C501B4010E948A31F6016193719388
:1034D000819391936F01FFEFEF1AFF0AE8CF61E04C
:1034E00072E0CE0101960E942513BE016F5F7F4FEF
:1034F0008AEB95E00E949C11182FCE0101960E9444
:103500000212112309F44BCA43E050E06AEB75E064
:10351000CE0145960E948213BE016B5E7F4FCE01A5
:1035200001960E941C1360E0CE0101960E94671272
:10353000BC0188EA95E00E940513CE0101960E9425
:103540000212CE0145960E94021268EA75E0CE0191
:103550008F960E941C1365E072E0CE0101960E94D6
:1035600025138BA99CA9892BC9F10FA518A96981DD
:103570007A81C8010E944D38009781F19C01201B7F
:10358000310B8901CE0101960E9402126BE571E0B8
:10359000CE0189960E9425136BE571E0CE018396DA
:1035A0000E94251310161106E4F467E072E0CE01C4
:1035B00001960E942513CE0101960E948E13CE0122
:1035C00001960E940212CE0183960E940212CE0141
:1035D00089960E940212CE018F969ACC0FEF1FEFB0
:1035E000D1CFBE01615D7F4FCE0183960E9405134E
:1035F000D12CC12C8AEF682E77247A9496E0592E2C
:103600008FA198A5009709F409C135E0C316D1042C
:10361000C9F368ED72E0CE0101960E942513BE0148
:103620006F5F7F4FCE0183960E949C11182FCE01B1
:1036300001960E9402121111CAC001E010E0980127
:1036400050E040E0BE016D5D7F4FCE0145960E9487
:103650003613BE016B5E7F4FCE0101960E941C1394
:1036600060E0CE0101960E946712BC01CE018996EE
:103670000E940513CE0101960E940212CE014596CA
:103680000E940212BE01675D7F4FCE0145960E94E7
:103690001C13898D9A8D029708F49CC068ED72E026
:1036A000CE0101960E942513BE016F5F7F4FCE01B0
:1036B00045960E949C11F82ECE0101960E9402129E
:1036C000FF2009F487C022E030E041E050E0BE0175
:1036D0006B5E7F4FCE0101960E943613CE0101969C
:1036E0000E9491114B017B01CE0101960E940212B2
:1036F00097FE03C04CE1E40EF11CB3016E197F0983
:103700005C9C70015D9CF00C1124F701E159FA4FAB
:1037100076876587CE0145960E940212B7016858E8
:103720007A4F44E050E0CE0189960E941F118FEF3E
:10373000C81AD80A8FA198A50817190708F067C0FA
:10374000A801BE016D5D7F4FCE0101960E948213DC
:10375000BE016F5F7F4FCE0189960E94B711CE01E7
:1037600001960E940212BE01675D7F4FCE018396D3
:103770000E940513ABA0BCA0A114B10409F440CF72
:103780000FA118A575010115110509F439CF4701DD
:103790009FEF891A990AF7018081082E000C990B76
:1037A0000E94CB2F892BD9F4015011090A0D1B1D42
:1037B000F8018081082E000C990B0E94CB2F892BD9
:1037C00081F00E151F0568F001501109F1CF02E0DC
:1037D00010E035CFCE0145960E94911191CF740132
:1037E000D6CF0F5F1F4FA8014E195F0958A74FA3EF
:1037F000AE14BF0420F4B701C5010E942038EBA12C
:10380000FCA18FA198A5E80FF91F1082F9CE6BE5F6
:1038100071E0CE0183960E94CF12F2CEC092710564
:10382000CC2041F081E080936F058EE190E00E9412
:103830006D14C9CE10926F05F8CF80E044C92F9265
:103840003F924F925F926F927F928F929F92AF9230
:10385000BF92CF92DF92EF92FF920F931F93CF937D
:10386000DF93CDB7DEB7C854D1090FB6F894DEBFE9
:103870000FBECDBF8C016BE571E080EC95E00E943E
:10388000CF12C8010596059760F08091F70381116A
:1038900008C00C3E2FEF120724F01093F2030093A0
:1038A000F103F8017A96E432F10508F0AAC7E55A67
:1038B000F34E0C94DC348E2301248A23012401244A
:1038C000012401240124012401240124AF1CAF1C84
:1038D000AF1C7F1CB81EAF1CB41F8820AF1CAF1CD0
:1038E000BB21CA21CD210124AF1CAF1CAF1CDB21A1
:1038F000D22263238023AF1CAF1CAF1CAF1C8E01F0
:10390000005E1F4F6FE0C8010E94E00518870F831B
:103910001D821E82198289E08A8381E08B838C83D9
:103920001C8A1B8ACE0101960E94640FCE0101966B
:103930000E94EC04CE0101960E941110EE80F12C41
:1039400035E0E316F1040CF0F6C0E114F10409F0DF
:10395000F5C069E675E080EC95E00E940513809162
:10396000C4059091C505892B09F4C5C060EC75E0CC
:10397000CE0101960E941C13CE0101960E948E1367
:10398000CE0101960E94021260EC75E0CE01809695
:103990000E941C1380913803882309F4A8C08091E9
:1039A0005D0390915E03843191050CF0A0C00091FD
:1039B000040110910501013CF3E01F070CF097C0D2
:1039C000019690935E0380935D030E94EB03C09089
:1039D0003003D0903103E0903203F09033036C1940
:1039E0007D098E099F090E94013020E030E04AE7FE
:1039F00054E40E94F731609334037093350380934D
:103A0000360390933703083C110534F488EC90E0BA
:103A10009093050180930401809104019091050128
:103A200028E3C22E23E0D22E04E313E09C012453AA
:103A300033407901C701800F911F9A838983D80190
:103A40006D918D01CE0101960E942B14C016D106F6
:103A500089F7E0900401F0900501C7010496909366
:103A6000050180930401BE01605E7F4FCE01019687
:103A70000E941C1360E0CE0101960E946712BC01F7
:103A800080EC95E00E940513CE0101960E9402127F
:103A90004091C4055091C5054115510531F069E3C8
:103AA00073E080EC95E00E941F118DE5C82E83E045
:103AB000D82E09E313E0F701E553F3407F01C70176
:103AC000800F911F9A838983D8016D918D01CE015A
:103AD00001960E942B14C016D10689F7809104012B
:103AE0009091050184969093050180930401CE0185
:103AF00080960E94021264E670E080E090E00E94EE
:103B00005F03C85BDF4F0FB6F894DEBF0FBECDBFBB
:103B1000DF91CF911F910F91FF90EF90DF90CF90A9
:103B2000BF90AF909F908F907F906F905F904F90DD
:103B30003F902F900895B4E0EB2EF12C6BE571E0EF
:103B400080EC95E00E94CF12A7E4CA2EA5E0DA2E01
:103B500010E000E0602FCE0101960E94F80E4B01AC
:103B60005C01D6014D905D906D907D906D01A3013B
:103B70009201C301B2010E944833811108C0A30120
:103B80009201C501B4010E948B314B015C010F5FB2
:103B90001F4F20E030E04CEF52ECC501B4010E9411
:103BA000FC2F87FF25C0B801CE01C4960E94D91210
:103BB00069E871E0CE018E960E942513BE016C5C0F
:103BC0007F4FCE018E960E949B126EE771E00E949D
:103BD000851269E675E00E949B120E945E12CE017A
:103BE0008E960E940212CE01C4960E94021272C0EA
:103BF000B3E0EB16F10409F49FC0B801CE01C496FE
:103C00000E94D91269E871E0CE018E960E942513B8
:103C1000BE016C5C7F4FCE018E960E949B12BC0150
:103C200082EA95E00E940513CE018E960E94021250
:103C3000CE01C4960E94021222E0B501A401CE0179
:103C4000C4960E94F51362EA75E0CE018E960E943A
:103C50001C1367E772E0CE018E960E948512BE01AA
:103C60006C5C7F4F0E949B12BC0182EA95E00E942F
:103C70000513CE018E960E940212CE01C4960E94B8
:103C8000021260EC75E0CE018E960E941C1362EA6F
:103C900075E0CE018E960E949B12BC0180EC95E0EF
:103CA0000E940513CE018E960E94021260EC75E010
:103CB000CE018E960E941C1360E2CE018E960E9469
:103CC0006712BC0180EC95E00E940513CE018E9630
:103CD0000E9402120E151F0509F03CCF033011059A
:103CE000A9F46EE172E0CE018E960E94251360EC7D
:103CF00075E0CE018E960E949B12BC0180EC95E08F
:103D00000E940513CE018E960E94021260EC75E0AF
:103D1000CE018E960E941C1368E272E0CE018E9650
:103D20000E948512BC0180EC95E00E940513CE0133
:103D30008E960E94021213CE22E0B501A401CE019C
:103D40008E960E94F513BE01625D7F4FCE01C49630
:103D50000E941C1360E2CE01C4960E9467120E946A
:103D60005E12CE01C4960E940212CE018E963DCF05
:103D700060E080E10E94EE028091F7038111E9C0CA
:103D80002AE030E040E050E029962CAF3DAF4EAF46
:103D90005FAF29976BE372E080EC95E00E94CF1251
:103DA000312C212C23961FAE239724961FAE2497E7
:103DB000C12CD12C760102E310E0812C912C54010E
:103DC00080E10E941F03092E000CAA0BBB0B880E7A
:103DD000991EAA1EBB1E65E070E080E090E00E9484
:103DE0005F030150110961F740904305509044056D
:103DF0006090450570904605C501B4010E940330EE
:103E000020E030E040EA50E40E94623020E030E000
:103E100040E85AE30E94623020E030E048E452E497
:103E20000E94F731A30192010E948A3120E030E024
:103E300040E751E40E9462304B015C01A301920112
:103E40006AE979E989E390E40E948A319B01AC0137
:103E5000C501B4010E94F73120E030E0A9010E94C1
:103E60008B3120E030E040E251E40E9462305B019F
:103E70008C01232D322D23964FAD239724965FADD1
:103E800024970E94F332181644F43A2C2B2C2396D4
:103E90000FAF239724961FAF24979FEFC91AD90A13
:103EA000E90AF90A29962CAD3DAD4EAD5FAD2997D3
:103EB0002C153D054E055F050CF07DCF6EE170E0E1
:103EC00080E090E00E945F0362E472E080EC95E0A5
:103ED0000E94CF1222E0432D522D23966FAD2397DF
:103EE00024967FAD2497CE0101960E94F513BE0162
:103EF0006F5F7F4FCE0180960E941C136FE472E0CB
:103F0000CE0180960E948512BC0188EA95E00E944D
:103F10000513CE0180960E940212CE0101960E94E6
:103F2000021266E572E0CE0101960E94251368EA4E
:103F300075E0CE0101960E949B1260EC75E00E9434
:103F40009B12BC0180EC95E00E940513CE01019606
:103F5000F0CE83E090E0A0E0B0E029968CAF9DAF7A
:103F6000AEAFBFAF299716CF68EC70E080E090E06D
:103F70000E945F030E94520A64E670E080E090E0D5
:103F80000E945F0362E370E080E090E00E945F03C4
:103F900049E050E064E171E084EF95E00E947C012B
:103FA00062E370E080E090E00E945F0303E010E0D5
:103FB00084EF95E00E948106892B61F149E050E091
:103FC00064E171E084EF95E00E947C0165E070E0BF
:103FD00080E090E00E945F03F12CE12C84EF95E0FB
:103FE0000E94810632E0E316F104A4F484EF95E028
:103FF0000E948106892B39F084EF95E00E94990692
:104000004FEFE41AF40A65E070E080E090E00E946F
:104010005F03E4CF62E370E080E090E00E945F0322
:104020000150110929F68AE090E00E94580A6B01BC
:104030007C0120E030E0A9010E94FC2F181634F02A
:104040008AE090E00E94580A6B017C010BE010E0CE
:1040500020E030E042ED53E4C701B6010E94FC2F9E
:10406000181684F00150110969F068EC70E080E0E6
:1040700090E00E945F0383E090E00E94580A6B0189
:104080007C01E6CF20E030E0A901C701B6010E9423
:10409000FC2F18160CF05DCC20E030E048EC52E428
:1040A000C701B6010E94FC2F21E087FF20E0B70185
:1040B000A601CE0101960E94F513BE016F5F7F4FEE
:1040C00080EC95E00E94B711CE0101960E94021289
:1040D00060EC75E0CE0101960E941C136AE572E067
:1040E000CE0101960E948512BC0180EC95E00E94F1
:1040F0000513CE0101960E9402126EE572E0CE0118
:1041000001960E94251360EC75E0CE01019617CF51
:104110000E94EB034B015C0184EF95E00E94EC06EA
:1041200064E670E080E090E00E945F030E94020776
:1041300064E670E080E090E00E945F0323961FAE8B
:104140002397D12CC12C312C212C25961FAE1EAECD
:104150002597FCED4F2EF5E05F2E612C712CCE01E2
:10416000809622969FAF8EAF22970E94EB0368192C
:1041700079098A099B09683B7B408105910508F014
:104180006BC084EF95E00E948106892B09F451C031
:104190004092F8055092F9056092FA057092FB057D
:1041A0000E94BA0697FD45C082349105C9F78E0179
:1041B0000F5F1F4F78010E94BA0697FF41C08981A7
:1041C0008D34B9F59801235E3F4F90E080E0D8012F
:1041D0004D918D01840F911DA217B307C1F78E5B1E
:1041E0009F4F2E8D30E0322F22274F8D240F311D0F
:1041F00082179307F1F48C8190E0982F88272D8106
:10420000FC01E20FF11D2596FFAFEEAF25972E8042
:10421000312C322C22248F81280E311CC884D12CC1
:10422000DC2CCC248985C80ED11CF1E02396FFAF8D
:10423000239762E370E080E090E00E945F0395CFF7
:10424000F70181937F0122962EAD3FAD22972E1765
:104250003F0709F0B0CFB3CF0E94EB03681979098B
:104260008A099B09683B7B4081059105A8F4239648
:104270003FAD2397332309F477C062E370E080E019
:1042800090E00E945F0384EF95E00E94EC0662E3F9
:1042900070E080E090E07BC023964FAD23974423ED
:1042A00009F462C0B601CE0180960E94D912B10114
:1042B000CE018E960E94D91225966EAD7FAD2597C0
:1042C000CE01CA960E94D912BE01665C7F4FCE0114
:1042D000C4960E941C1364E572E0CE01C4960E944D
:1042E0008512BE01625D7F4F0E949B1264E572E001
:1042F0000E948512BE01605E7F4F0E949B1263E6A2
:1043000072E00E948512BC0188EA95E00E940513C4
:10431000CE01C4960E940212CE01CA960E940212D9
:10432000CE018E960E940212CE0180960E94021249
:1043300069E672E080EC95E00E94CF1260EC75E0D7
:10434000CE0180960E941C1368EA75E0CE0180962B
:104350000E949B12BC0180EC95E00E940513CE01E7
:1043600080960E94021289CF69E675E080EC95E0A4
:104370000E94051382CF8091F703882321F080ECFF
:1043800095E00E94A90168EC70E080E090E00E9456
:104390005F03E5CA1092F703E2CA81E08093F70356
:1043A000809377058091F1039091F2039093F0034D
:1043B0008093EF03D4CA80910701882309F4CFCA00
:1043C0000E943E0C2B013C010E94B00B4B015C0192
:1043D00060912705709128058091290590912A0503
:1043E0000E94033020E030E048EC52E40E94F731B4
:1043F0006B017C010E943E0C20E030E048EC52E46E
:104400000E94F731A70196010E94F73121E03EEDAD
:1044100042E45EE30E94F8326B017C0120E030E070
:1044200048EC52E4C301B2010E94F731AB01BC0178
:1044300022E0CE0180960E94F513BE01605E7F4FA0
:10444000CE0101960E941C1369E772E0CE0101962D
:104450000E948512BC0182EA95E00E940513CE01FC
:1044600001960E940212CE0180960E94021262EA18
:1044700075E088EA95E00E9405136FEB71E0CE01CC
:1044800001960E94251362EA75E0CE0101960E9412
:104490009B12BC0182EA95E00E940513CE010196B1
:1044A0000E94021221E0B501A401CE0180960E9473
:1044B000F513BE01605E7F4FCE0101960E941C1372
:1044C0006EE772E0CE0101960E948512BC0180EC7D
:1044D00095E00E940513CE0101960E940212CE01C2
:1044E00080960E94021269EB71E0CE0101960E9453
:1044F000251360EC75E0CE0101960E949B1261E8E5
:1045000072E00E948512BC0180EC95E00E940513C8
:10451000CE0101960E940212A701960160E070E0B0
:1045200080E89FE30E948A3120E03AE24DE257E4BE
:104530000E946230AB01BC0121E0CE0180960E9456
:10454000F513BE01605E7F4FCE0101960E941C13E1
:104550006CE572E0CE0101960E9485120E945E1207
:10456000CE0101960E940212CE0180960E94021294
:1045700062EA75E0CE0101960E941C1360EC75E0C2
:10458000CE0101960E949B12BC0180EC95E00E9436
:104590000513CE0101960E94021265E070E080E0F2
:1045A00090E0F5CE3BE0C32ED12C10E000E0992442
:1045B000939443E2842E90924E0480927004109261
:1045C0004F041092710462E083E20E94FB08109293
:1045D0000104809300048FE095E00E94D909F82E31
:1045E000E12C8FE095E00E94D9095C01AE28BF283C
:1045F0000E941408B50190E080E00E9401302AE991
:1046000039E949E95FE30E94F7310E9470320617E9
:10461000170708F48B0162E370E080E090E00E94ED
:104620005F0351E0C51AD10831F665E872E080EC0D
:1046300095E00E94CF1219A218A21BA21AA21DA2D5
:104640001CA24AE0BE016F5F7F4FC8010E942A2C66
:10465000BE016F5F7F4FCE0180960E94CF12BE01D8
:10466000605E7F4FCE0101960E941C1365E972E0E7
:10467000CE0101960E948512BC0188EA95E00E9455
:104680000513CE0101960E940212CE0180960E946F
:1046900002126AE972E0CE0101960E94251368EACF
:1046A00075E0CE0101960E949B1260EC75E00E94BD
:1046B0009B12BC0180EC95E00E940513CE0101968F
:1046C0000E940212E4CD81E0809306010E949203D1
:1046D0008C016DE972E080EC95E00E94CF1260E001
:1046E00074E0601B710BCE0101960E94D912CE01BD
:1046F00001960E945E12CE0101960E9402122FC9FD
:104700006DEA72E080EC95E00E94CF120E94920365
:10471000BC01E9CFF0E0E0E0099521C98091710585
:1047200018160CF055C081E080936F0568EB72E0BD
:1047300080EC95E00E94CF1280916F05882309F4E8
:104740004AC066EC72E0CE0101960E94251360EC2F
:1047500075E0CE0101960E949B12BC0180EC95E0B1
:104760000E940513CE0101960E94021260EC75E0D2
:10477000CE0101960E941C13CE0101960E948E1359
:10478000CE0101960E94021268EE73E080E090E094
:104790000E945F0380916F0581110E9408246BE5E0
:1047A00071E080EC95E00E94CF128091F703809336
:1047B00077058111D4C867ED72E084EB95E00E9423
:1047C000CF1286EE9FEF9093F2038093F103C7C858
:1047D00010926F05ABCF6EEC72E0CE0101960E9495
:1047E000251360EC75E0CE0101960E949B12BC017E
:1047F00080EC95E00E940513CE0101960E94021202
:10480000D4CF6AED72E080EC95E00E94CF12A7C889
:104810000F931F93CF93DF930FE615E0D0E0C0E036
:104820000A5F1F4F80917105082E000C990BC81765
:10483000D9076CF4F801878190850E941F1C68EEEF
:1048400073E080E090E00E945F032196E9CFDF9162
:10485000CF911F910F9108951F920F920FB60F9253
:1048600011242F933F934F935F936F937F938F9375
:104870009F93AF93BF93EF93FF9382E794E00E94DF
:104880001302FF91EF91BF91AF919F918F917F9113
:104890006F915F914F913F912F910F900FBE0F90AD
:1048A0001F9018951F920F920FB60F9211242F93FD
:1048B0008F939F93EF93FF93E0918204F091830491
:1048C0008081E0918804F091890482FD1BC0908171
:1048D00080918B048F5F8F7320918C04821741F03D
:1048E000E0918B04F0E0EE58FB4F958F80938B04A2
:1048F000FF91EF919F918F912F910F900FBE0F908D
:104900001F9018958081F4CF1F920F920FB60F92CF
:1049100011242F933F938F939F93AF93BF938091D5
:10492000E4039091E503A091E603B091E703309191
:10493000E30323E0230F2D3758F50196A11DB11D88
:104940002093E3038093E4039093E503A093E603AD
:10495000B093E7038091E8039091E903A091EA0303
:10496000B091EB030196A11DB11D8093E8039093D4
:10497000E903A093EA03B093EB03BF91AF919F913A
:104980008F913F912F910F900FBE0F901F90189510
:1049900026E8230F0296A11DB11DD2CF1F920F92C0
:1049A0000FB60F9211242F933F934F935F936F9302
:1049B0007F938F939F93AF93BF93EF93FF93E09178
:1049C000FE03F091FF03309749F0A685B7858585F2
:1049D000968D91FF14C09C918923A1F4FF91EF91D2
:1049E000BF91AF919F918F917F916F915F914F9107
:1049F0003F912F910F900FBE0F901F9018959C9193
:104A0000892361F7A389B4899C918589809589233D
:104A10008C93868997890197F1F7608D718DA685B2
:104A2000B785558538E020E0CB010197F1F7822F5B
:104A300090E095958795282F4C91452309F02068A3
:104A4000315091F7868D81FD20958091FD0390E096
:104A500001968F7399273091FC03381799F0A09134
:104A6000FD03B0E0AD55BC4F2C938093FD03828DC8
:104A7000938D0197F1F7A389B4898C919589892B3E
:104A80008C93ACCF868D8160868FF1CF1F920F9271
:104A90000FB60F9211242F933F934F935F936F9311
:104AA0007F938F939F93AF93BF93EF93FF938091E7
:104AB000B900887F803609F44AC0F0F5883209F4DD
:104AC000A7C018F5803109F49BC0B8F4882309F415
:104AD000F9C0883009F494C0FF91EF91BF91AF9174
:104AE0009F918F917F916F915F914F913F912F9106
:104AF0000F900FBE0F901F901895883109F488C051
:104B0000803251F78093460414C0803409F49DC06C
:104B100040F48033B9F38833F9F68093460485EC8A
:104B2000B0C0803509F485C0883509F496C0883452
:104B300099F60E945911D0CF883909F48CC038F504
:104B4000883729F050F4883611F0803729F683E051
:104B5000809348041092A20357C0883809F47BC0A0
:104B6000803919F0803809F0B7CF8091A2038032E4
:104B700008F071C0E091A20381E08E0F8093A20340
:104B80008091BB00F0E0EE57FC4F80833DC0803B3E
:104B900039F0E0F4803A09F479C0883A09F09CCF02
:104BA00084E0809348041092810310928003E09186
:104BB000FA03F091FB0309958091800381110FC0E6
:104BC00081E0809380031092600309C0803C09F467
:104BD000A6CF883C09F4A3CF883B09F07DCFE091B4
:104BE000810381E08E0F80938103F0E0E05AFC4F57
:104BF00080818093BB00909181038091800329C0C4
:104C0000809123048093BB0085EC8093BC0064CF2B
:104C10009091450480914404981758F5E09145041B
:104C200081E08E0F80934504F0E0EC5DFB4F8081C6
:104C3000E9CFE091450481E08E0F80934504809197
:104C4000BB00F0E0EC5DFB4F8083909145048091C8
:104C500044049817C8F285E8D8CFE091450481E074
:104C60008E0F809345048091BB00F0E0EC5DFB4F1C
:104C700080838091470481115CCF81E0809322047E
:104C800084EA8093BC001092480426CF85EC809380
:104C9000BC00109248048091A203803230F4E0916D
:104CA000A203F0E0EE57FC4F10826091A20370E087
:104CB000E091F803F091F90382E893E009951092EE
:104CC000A2030ACF1092460434CF8091A805909198
:104CD000A905009711F00C94DF2B60E070E0CB0188
:104CE0000895109275041092740488EE93E0A0E089
:104CF000B0E08093760490937704A0937804B09307
:104D0000790427E231E0309373042093720425EC98
:104D100030E030937F0420937E0424EC30E0309325
:104D200081042093800420EC30E0309383042093AE
:104D3000820421EC30E0309385042093840422EC3B
:104D400030E0309387042093860426EC30E03093E3
:104D500089042093880410928B0410928C04109282
:104D60008D0410928E0410921205109211058093FA
:104D7000130590931405A0931505B093160529E328
:104D800031E03093100520930F051092F705109233
:104D9000F6058093F8059093F905A093FA05B09372
:104DA000FB058BE491E09093F5058093F405109258
:104DB0000B0610920A0610920D0610920C06109225
:104DC0000F0610920E0610921106109210066091B6
:104DD00012066E7F6D7F609312066695617081E0AA
:104DE000682789E00E94A20261E089E00E94EE0249
:104DF000EEE8F2E0E491E0930406EAE7F2E0E49101
:104E0000F0E0EE0FFF1FE959FD4F859194919093CB
:104E100006068093050660E08AE00E94EE0280911B
:104E2000120681FD04C061E08AE00E94A2028AE0CD
:104E300080930006EFE8F2E0E491E0930106EBE7EF
:104E4000F2E0E491F0E0EE0FFF1FE35AFD4F859191
:104E5000949190930306809302068FEF8093CF0581
:104E60008093D0058093D1058093D2056BE571E0E6
:104E700080EC95E00E9425136BE571E08AEB95E0EC
:104E80000E9425136BE571E084EB95E00E942513E9
:104E90006BE571E08EEA95E00E9425136BE571E009
:104EA00088EA95E00E9425136BE571E082EA95E0BF
:104EB0000E94251368EE72E08CE995E00E942513AC
:104EC0006FEE72E086E995E00E94251310926F055F
:104ED00085E0809370051092710510927305109211
:104EE0007205109275051092740510927605109255
:104EF00077056CEF72E089E695E00E94251386E164
:104F000090E090931C0580931B058CE79CE8A1E042
:104F1000B0E08093270590932805A0932905B093CE
:104F20002A0581EA97E6A3E3BDEB80932B059093D6
:104F30002C05A0932D05B0932E0586E696E6A6EAED
:104F4000BFE380932F0590933005A0933105B09374
:104F500032051092330510923405109235051092E7
:104F600036051092370510923805109239051092C7
:104F70003A0581E080933B0529E130E030933D051F
:104F800020933C0580933E0580E090E4ACE1B5E4DD
:104F900080933F0590934005A0934105B09342054F
:104FA0001092430510924405109245051092460553
:104FB000E7E4F5E080E1DF011D928A95E9F71092C0
:104FC0005705109258051092590510925A051092E3
:104FD0005B0510925C0510925D0510925E051092C3
:104FE0005F051092600510926105109262051092A3
:104FF000630510926405109265051092660581E0C4
:1050000090E090936805809367050895CF93DF93B0
:10501000CDB7DEB72C970FB6F894DEBF0FBECDBF6D
:10502000789484B5826084BD84B5816084BD85B583
:10503000826085BD85B5816085BD80916E0081608F
:1050400080936E0010928100809181008260809335
:105050008100809181008160809381008091800037
:105060008160809380008091B10084608093B10062
:105070008091B00081608093B00080917A0084605C
:1050800080937A0080917A00826080937A00809188
:105090007A00816080937A0080917A0080688093A2
:1050A0007A001092C10061E08EE00E94EE02E09171
:1050B0008204F091830482E08083E0917E04F09189
:1050C0007F041082E0918004F09181048FEC808352
:1050D00010928A04E0918604F091870486E0808330
:1050E000E0918404F0918504808180618083E09167
:1050F0008404F0918504808188608083E091840439
:10510000F0918504808180688083E0918404F0912F
:10511000850480818F7D808360E08EE00E94A20202
:105120000E94DC0781E080934E0483E28093700448
:1051300010924F041092710460E18FE095E00E949C
:10514000200A0E9414088FE39CE90197F1F700C040
:10515000000068EC70E080E090E00E945F0384E66D
:1051600090E090930901809308010E94233180937D
:10517000EC0385E690E00E9423318093ED030091DB
:10518000EC031091ED03B801012E000C880B990B74
:105190000E9403309B01AC010E944833811106C07C
:1051A0000B5011090C30110508F4EDC084E690E0B5
:1051B0000E9444143FE6C32E35E0D32E56010EE183
:1051C00010E0C8010E942331F50181935F010F5F58
:1051D0001F4F07321105A9F710917005612F012E9D
:1051E000000C770B880B990B0E9403309B01AC01DC
:1051F0000E944833811103C0153009F4E7C08EE1E5
:1052000090E00E946D1468EC70E080E090E00E94F5
:105210005F0368E073E080EC95E00E94CF120E948B
:10522000DC0764E670E080E090E00E945F036CE9D8
:1052300075E0CE0101960E941C1360E0CE0101963C
:105240000E9467120E945E12CE0101960E94021215
:1052500060EC75E0CE0101960E941C13CE01019610
:105260000E948E13CE0101960E94021286E780935F
:10527000C6058091CF058F3F11F40E94DC07809115
:10528000CF058F3F01F58091C60591E090934E04C4
:105290008093700410924F041092710460ED8FE0BF
:1052A00095E00E94200A0E94140861E08091C605E2
:1052B0000E94FB0810920104809300048FE095E0A7
:1052C0000E94D909F82EF8E5FF1609F48DC061E1B6
:1052D00073E080EC95E00E94CF121092070160EC21
:1052E00075E0CE0101960E941C13CE0101960E942A
:1052F0008E13CE0101960E9402128AE2C82ED12C92
:1053000098EE892E93E0992EA12CB12C20E0E22E6C
:1053100020E0F22E01E06BE571E0CE0107960E94DD
:10532000251310E082E794E00E94F3011816190695
:105330000CF0CBC01111C9C082E794E00E94D101EA
:105340008A3009F072C11091EE03112309F482C171
:105350008091B2059091B305892B09F474C16DE178
:1053600073E0CE0101960E942513BE01695F7F4F55
:10537000CE0101960E949B120E94A901CE010196C6
:105380000E94021260C14BE1C42E45E0D42E04E617
:1053900010E0C8010E942331F60181936F010F5F75
:1053A0001F4F023B1105A9F76DE175E0CE01019693
:1053B0000E942513BE016F5F7F4F8CE995E00E942C
:1053C000B711CE0101960E940212F4CE0EE110E058
:1053D000C8010E942331F60181936F010F5F1F4FB7
:1053E00005341105A9F70FCF88E80E94EE109093BD
:1053F000D4058093D3058AE80E94EE109093D605D9
:105400008093D5058CE80E94EE109093D805809388
:10541000D7058EE80E94EE109093DA058093D905A7
:1054200080E90E94EE109093DC058093DB0582E911
:105430000E94EE109093DE058093DD0584E90E94C2
:10544000EE109093E0058093DF0586E90E94EE1050
:105450009093E2058093E10588E90E94EE10909315
:10546000E4058093E3058AE90E94EE109093E60537
:105470008093E5058CE90E94EE109093E8058093F7
:10548000E7058EE90E94EE109093EA058093E90506
:105490008091CF058F3F09F030CF8091C60591E014
:1054A00090934E048093700410924F0410927104F4
:1054B00064EF8FE095E00E94200A6FE38FE095E0B3
:1054C0000E94200A0E94140818CF8B859C85892B86
:1054D00051F082E794E00E94820264E170E080E093
:1054E00090E00E945F03BE01695F7F4F8EEA95E006
:1054F0000E94B711CE0107960E9402126BE571E07F
:1055000080EC95E00E94CF128091B2059091B30596
:105510008130910509F0C6C06EEA75E08AEB95E02E
:105520000E9405130E9442116AEB75E0CE010196BC
:105530000E941C138D819E81892B09F4A5C0E981ED
:10554000FA81309709F4A0C08081823409F484C0C4
:10555000833409F48EC0813409F096C066E273E0AA
:105560008EEA95E00E94CF12CE0101960E940212AF
:105570008EEA95E00E949111CB010E941F1C809140
:10558000F703882309F43FC00E94EB03A5019401AF
:105590000E94BA34CA01B9010E9401302091F3037C
:1055A0003091F4034091F5035091F6030E948A3143
:1055B00020910A0130910B0140910C0150910D0195
:1055C0000E94F3321816FCF48091F1039091F203DB
:1055D0004A9609F4A0C08091EF039091F0030E94D5
:1055E0001F1C0E94EB03A50194010E94BA34CA015A
:1055F000B9010E9401306093F3037093F403809328
:10560000F5039093F6036AE070E080E090E00E947A
:105610005F03E114F10409F47ECE0E94FF018823A8
:1056200009F479CE0E94000076CE8D3009F48BCE3D
:1056300089831A8241E050E0BE016F5F7F4FCE0147
:1056400007960E9432126AE070E080E090E00E94CB
:105650005F0368CE11E0F7CF69E273E08EEA95E070
:105660000E94CF121092F7038CEF9FEF0E941F1C35
:105670007BCF6CE273E08EEA95E00E94CF1200933C
:10568000F7038DEF9FEFF2CFBE016F5F7F4F8EEA82
:1056900095E00E9405136AE070E080E090E00E94CF
:1056A0005F0362CF049768F568ED72E0CE01019662
:1056B0000E942513BE016F5F7F4F8EEA95E00E9426
:1056C0009C11182FCE0101960E9402121123C9F0DD
:1056D0008091B2059091B305029788F0E091AE05F4
:1056E000F091AF05309759F0818180330CF4845EDE
:1056F0009601281B310987FD3395C9013ECF80E013
:10570000F6CF8091B2059091B305029708F437CF98
:105710000E94961434CF80916F05882309F461CFDD
:105720000E9408245ECF89E695E00E94021286E975
:1057300095E00E9402128CE995E00E94021282EA32
:1057400095E00E94021288EA95E00E9402128EEA19
:1057500095E00E94021284EB95E00E9402128AEB0F
:1057600095E00E94021280EC95E00E9402128BE408
:1057700091E09093F5058093F40584EF95E00C9407
:10578000EC06EF920F931F93CF93DF93E80134E081
:1057900047FD34E1042E000C550B57FF03C0519513
:1057A00041955109E32E022F242FAE010E94442C73
:1057B000CE01DF91CF911F910F91EF900895662751
:1057C00077270C94A32D1F93FC0199278827BC01F0
:1057D000E89411911032E9F3193010F01E30C8F33B
:1057E0001B3251F01D3249F4689406C00E94152CFA
:1057F000610F711D811D911D119110531A30B0F36D
:105800003EF490958095709561957F4F8F4F9F4F97
:105810001F910895BB274A3031F4992322F4BDE249
:10582000909581959F4F0C942B2C592F482F372FF3
:10583000262F660F771F881F991F660F771F881FF7
:10584000991F620F731F841F951F660F771F881F94
:10585000991F0895BB27FB015527AA27880F991F79
:10586000AA1FA41710F0A41B83955051B9F7A05D8F
:10587000AA3308F0A95DA193009779F7B111B1930C
:105880001192CB010C94EC2FA9E0B0E0EAE4FCE229
:105890000C944A316A01F22EB02E102FFBE3AF2E8A
:1058A000A01608F41BE31F5F012F27E0AE014F5F36
:1058B0005F4F0E94F32EBC018981982F997091301F
:1058C00009F43FC09BE2E1FC04C09E2D9170E0FC16
:1058D0003AC05E2D5071E82FE87083FF46C084E027
:1058E000911101C083E0EF2DE81B8F1508F0E0E077
:1058F000D6018E2F20E2552351F1992329F0D601AC
:105900009C93C60101966C0196012D5F3F4FE2FE0C
:1059100024C08EE4D6018C9391E411969C93119748
:1059200012968C93D9018E2F90E281111BC0E20F49
:10593000F32FF11D10828EEF9FEF2996ECE00C946F
:1059400066319DE2C6CF90E2C4CF2D938150811184
:10595000FCCFCE0ED11CE0E0D0CF8EE6D6018C93EA
:1059600091E6DBCF9D938150E0CF482F447082FFBA
:105970003DC084E0911101C083E08F1510F4EF2D3C
:10598000E81BD6018E2F20E2552309F1992329F037
:10599000D6019C93C60101966C0196012D5F3F4F85
:1059A000E2FE1BC089E4D6018C938EE411968C93A1
:1059B000119786E412968C93D9018E2F90E288235A
:1059C00009F4B5CF9D938150FACF2D938150811169
:1059D000FCCFCE0ED11CE0E0D9CF89E6D6018C9366
:1059E0008EE611968C93119786E6E4CF9B0177FFA4
:1059F00002C030E020E0A1E0B0E0911102C0B0E0D0
:105A0000A0E0F9013196AE0FBF1F8B2C912CBB206B
:105A100009F461C05401EFEFAE1ABE0AAA0DBB1D16
:105A2000FA161B0619F014F04F2D4A1B511188C0AD
:105A3000E3FC59C07601A42FB0E2A1114FC0C40EFF
:105A4000D11C992309F45BC040E0D6011196F60100
:105A500090836D01552309F448C0012F060F9A81E8
:105A6000582F507184FF03C0913309F40150101670
:105A70000CF047C0093008F008E0EEE2FE2E5B01B2
:105A8000A01AB10885019194819491082F3F3207A3
:105A900029F4D601FC92F60131966F016217730763
:105AA00094F1021713077CF5DB01A21BB30BAA24A8
:105AB000A394B12CAC0EBD1EAA0DBB1D11968C91EA
:105AC00021503109D601119628153905F4F0F60157
:105AD00080836D01DBCFB12CA12CA0CFF701B19356
:105AE0007F01A150AACF9111B0CFD601942F50E3DE
:105AF00002C05D9391509111FCCFC40ED11C40E0C7
:105B0000ACCF01E0BACF80E3DBCF6217730731F48B
:105B1000963388F4953311F4552369F0F6018083A8
:105B2000FD01842F90E2811108C0A40FB11D1C92C9
:105B300090E080E002CF81E3F1CF91938150F3CFE9
:105B4000911183CF8ACFB0E0A0E0E9EAFDE20C94A6
:105B50004A315C017B016115710519F0DB018D9300
:105B60009C9385010F5F1F4FF501D0818D2F90E031
:105B70000E94CB2F6C01892BB9F5DD32B9F50F5F8F
:105B80001F4FD5011196DC91C1E05801F1E0AF1A29
:105B9000B10843E050E062EF70E0C5010E94D42FED
:105BA000892B69F5680182E0C80ED11C45E050E000
:105BB0006DEE70E0C6010E94D42F892B21F468019C
:105BC00097E0C90ED11CE114F10419F0D701CD9270
:105BD000DC9260E070E080E89FEFC111FFC060E000
:105BE00070E080E89FE7FAC05801BBCFDB3229F4B0
:105BF00085010E5F1F4FF501D181C0E0C6CF43E0A4
:105C000050E06AEE70E0C5010E94D42F892BE9F0C4
:105C1000F80110E000E020E030E0A9015F01B0ED04
:105C20008B2E8D0E89E08815C8F19C2E689491F812
:105C30008C2F8870C2FF16C0811102C00F5F1F4FEA
:105C40003196D501DC91C92DE9CFE114F10429F099
:105C50000E5F1F4FF7011183008360E070E080EC5E
:105C60009FE7BCC0882311F001501109A5E0B0E006
:105C70000E9439319B01AC01220F331F441F551F75
:105C8000280D311D411D511D283999E93907490752
:105C900099E15907A8F2C6609C2ED2CFAEEF8A12C6
:105CA00006C0C3FD3CC09C2E689493F8C9CFDF7D2D
:105CB000D534A9F580818D3239F4C061DF011296A7
:105CC000818162E070E006C0DF018B32C1F3119682
:105CD00061E070E080535D01A61AB70A8A30F8F4DB
:105CE000E0E8CE16ECE0DE065CF4B601660F771F46
:105CF000660F771FC60ED71ECC0CDD1CC80ED11C3C
:105D00005D01FFEFAF1ABF0A8C9180538A30A8F172
:105D1000C4FF03C0D194C194D1080C0D1D1DC1FF57
:105D200009C0E114F10431F081E0A81AB108D701EB
:105D3000AD92BC92CA01B9010E940130C370C33058
:105D400009F490584B015C0120E030E0A9010E9469
:105D5000FC2F882309F440C0C1E2D1E017FF05C041
:105D6000119501951109C9E0D1E06E01B8E1CB1A96
:105D7000D10880E2E82EF12C0FC0D501B1CFFE0191
:105D800025913591459154910E191F09C501B40112
:105D90000E9462304B015C01D501C4010E151F0544
:105DA00074F72497F594E794CC16DD06A9F78A2FAB
:105DB000880F8B2F881F8F3F49F020E030E0A9012A
:105DC000C501B4010E94FC2F811106C082E290E05F
:105DD0009093140680931306C501B401CDB7DEB7C6
:105DE000ECE00C946631283008F027E03327DA0124
:105DF000990F311D87FD916000966105710539F499
:105E000032602E5F3D9330E32A95E1F708959F3F7E
:105E100030F080387105610509F03C5F3C5F3D93CF
:105E2000913008F08068911DDF93CF931F930F93FB
:105E3000FF92EF92192F987F9695E92F9695969558
:105E4000E90FFF27E158FE4F99273327EE24FF245F
:105E5000A701E70105900894079428F4360FE71E80
:105E6000F81E491F511D660F771F881F991F069442
:105E7000A1F70590079428F4E70EF81E491F561F56
:105E8000C11D770F881F991F661F0694A1F7059003
:105E9000079428F4F80E491F561FC71FD11D880FFD
:105EA000991F661F771F0694A1F70590079420F4A9
:105EB000490F561FC71FD81F990F661F771F881FCE
:105EC0000694A9F784911095177041F0D695C7955F
:105ED00057954795F794E7941A95C1F7E5E2F1E0F5
:105EE00068941590159135916591959105907FE293
:105EF0007395E118F10A430B560BC90BD009C0F793
:105F0000E10CF11E431F561FC91FD01D7EF47033D4
:105F100011F48A95E6CFE894015030F0080F0AF4A6
:105F20000027021708F4202F2395022F7A3328F038
:105F300079E37D932A95E9F710C07D932A9589F638
:105F4000069497956795379517951794E118F10A78
:105F5000430B560BC90BD00998F023957E9173958E
:105F60007A3308F070E37C932013B8F77E91706168
:105F70007D9330F0839571E37D9370E32A95E1F78B
:105F80001124EF90FF900F911F91CF91DF919927EE
:105F900087FD9095089591110C94CF30803219F0BF
:105FA00089508550C8F70895FB01DC0141505040ED
:105FB00088F08D9181341CF08B350CF4805E6591F6
:105FC00061341CF06B350CF4605E861B611171F35B
:105FD000990B0895881BFCCFDC01FC01672F7191A0
:105FE0007723E1F7329704C07C916D9370836291BF
:105FF000AE17BF07C8F308950E943E3008F481E051
:106000000895E89409C097FB3EF4909580957095AB
:1060100061957F4F8F4F9F4F9923A9F0F92F96E9F4
:10602000BB279395F695879577956795B795F11169
:10603000F8CFFAF4BB0F11F460FF1BC06F5F7F4F06
:106040008F4F9F4F16C0882311F096E911C0772318
:1060500021F09EE8872F762F05C0662371F096E821
:10606000862F70E060E02AF09A95660F771F881FF0
:10607000DAF7880F9695879597F90895990F000894
:10608000550FAA0BE0E8FEEF16161706E807F9070A
:10609000C0F012161306E407F50798F0621B730BA5
:1060A000840B950B39F40A2661F0232B242B252B26
:1060B00021F408950A2609F4A140A6958FEF811DC9
:1060C000811D08950E9475300C94E9300E94DB30E8
:1060D00038F00E94E23020F0952311F00C94D23079
:1060E0000C94D83011240C941D310E94FA3070F3B6
:1060F000959FC1F3950F50E0551F629FF001729F6D
:10610000BB27F00DB11D639FAA27F00DB11DAA1F7B
:10611000649F6627B00DA11D661F829F2227B00DC8
:10612000A11D621F739FB00DA11D621F839FA00D53
:10613000611D221F749F3327A00D611D231F849FA3
:10614000600D211D822F762F6A2F11249F575040FA
:106150009AF0F1F088234AF0EE0FFF1FBB1F661F75
:10616000771F881F91505040A9F79E3F510580F03E
:106170000C94D2300C941D315F3FE4F3983ED4F37D
:10618000869577956795B795F795E7959F5FC1F7E2
:10619000FE2B880F911D9695879597F9089599275D
:1061A0008827089597F99F6780E870E060E0089578
:1061B0009FEF80EC089500240A941616170618061F
:1061C0000906089500240A941216130614060506FB
:1061D0000895092E0394000C11F4882352F0BB0F8C
:1061E00040F4BF2B11F460FF04C06F5F7F4F8F4FEF
:1061F0009F4F089557FD9058440F551F59F05F3F2A
:1062000071F04795880F97FB991F61F09F3F79F0D8
:1062100087950895121613061406551FF2CF46955A
:10622000F1DF08C0161617061806991FF1CF8695DC
:106230007105610508940895E894BB2766277727C0
:10624000CB0197F90895F999FECF92BD81BDF89AD7
:10625000992780B50895262FF999FECF1FBA92BDD0
:1062600081BD20BD0FB6F894FA9AF99A0FBE019637
:1062700008950E947B31A59F900DB49F900DA49F1F
:10628000800D911D112408952F923F924F925F929D
:106290006F927F928F929F92AF92BF92CF92DF9236
:1062A000EF92FF920F931F93CF93DF93CDB7DEB79B
:1062B000CA1BDB0B0FB6F894DEBF0FBECDBF09942F
:1062C0002A88398848885F846E847D848C849B8486
:1062D000AA84B984C884DF80EE80FD800C811B8194
:1062E000AA81B981CE0FD11D0FB6F894DEBF0FBEC3
:1062F000CDBFED010895A29FB001B39FC001A39F40
:10630000700D811D1124911DB29F700D811D1124EE
:10631000911D08955058BB27AA270E94A2310C94C2
:10632000E9300E94DB3038F00E94E23020F039F48E
:106330009F3F19F426F40C94D8300EF4E095E7FB57
:106340000C94D230E92F0E94FA3058F3BA17620742
:1063500073078407950720F079F4A6F50C941C3197
:106360000EF4E0950B2EBA2FA02D0B01B901900170
:106370000C01CA01A0011124FF27591B99F0593FB4
:1063800050F4503E68F11A16F040A22F232F342FFC
:106390004427585FF3CF469537952795A795F0404A
:1063A0005395C9F77EF41F16BA0B620B730B840B5F
:1063B000BAF09150A1F0FF0FBB1F661F771F881F17
:1063C000C2F70EC0BA0F621F731F841F48F487956F
:1063D00077956795B795F7959E3F08F0B0CF939561
:1063E000880F08F09927EE0F9795879508950E94DA
:1063F0000B320C94E9300E94E23058F00E94DB30FE
:1064000040F029F45F3F29F00C94D23051110C94E4
:106410001D310C94D8300E94FA3068F39923B1F3FF
:10642000552391F3951B550BBB27AA2762177307BA
:10643000840738F09F5F5F4F220F331F441FAA1F4E
:10644000A9F335D00E2E3AF0E0E832D0915050400A
:10645000E695001CCAF72BD0FE2F29D0660F771FB8
:10646000881FBB1F261737074807AB07B0E809F09E
:10647000BB0B802DBF01FF2793585F4F3AF09E3F23
:10648000510578F00C94D2300C941D315F3FE4F349
:10649000983ED4F3869577956795B795F7959F5F66
:1064A000C9F7880F911D9695879597F90895E1E0B2
:1064B000660F771F881FBB1F621773078407BA0711
:1064C00020F0621B730B840BBA0BEE1F88F7E0956C
:1064D00008950E9470326894B1110C941D31089592
:1064E0000E94023188F09F5798F0B92F9927B75131
:1064F000B0F0E1F0660F771F881F991F1AF0BA9568
:10650000C9F714C0B13091F00E941C31B1E0089578
:106510000C941C31672F782F8827B85F39F0B93F6A
:10652000CCF3869577956795B395D9F73EF490951A
:106530008095709561957F4F8F4F9F4F089597FB82
:1065400016F40E94E3320C94A632E894F92F96EBED
:10655000FF2381F0121613061406440B9395F6954B
:1065600087957795679557954040FF23B9F71BC0EE
:1065700099270895882351F49850D2F7872B762FC6
:10658000652F542F432F322F20E0B1F3121613063C
:106590001406440B88233AF09A95440F551F661F42
:1065A000771F881FCAF755234AF4440F551F11F46B
:1065B00060FF04C06F5F7F4F8F4F9F4F880F96958E
:1065C000879597F908959095809570956095509569
:1065D0004095309521953F4F4F4F5F4F6F4F7F4F05
:1065E0008F4F9F4F08950E943E3008F48FEF08951B
:1065F000FA01EE0FFF1F309621053105A1F161155B
:10660000710561F48038BFE39B0749F168949038C5
:10661000810561F08038BFEF9B0741F099234AF56F
:10662000FF3FE1053105210519F1E8940894E7954C
:10663000D901AA2329F4AB2FBE2FF85FD0F310C0E5
:10664000FF5F70F4A695E0F7F73950F019F0FF3AC4
:1066500038F49F779F930DD00F9007FC90580895C2
:1066600046F00C94D83060E070E080E89FE3089535
:106670004FE79F775F934F933F932F930E94F83399
:106680002F913F914F915F910E9462300C9455334E
:106690000E943E30880B990B089529F416F00C9453
:1066A000D2300C941C310C94D8300E940231A8F3E3
:1066B0009638A0F707F80F92E8942BE33AEA48EBF4
:1066C0005FE70E9478300F920F920F924DB75EB73E
:1066D0000F920E944034E8E6F0E00E9487334F9129
:1066E0005F91EF91FF91E595EE1FFF1F49F0FE5777
:1066F000E0684427EE0F441FFA95E1F74195550BEA
:106700000E94BA330F9007FE0C94AE330895DF93C6
:10671000CF931F930F93FF92EF92DF927B018C0137
:10672000689406C0DA2EEF010E947530FE01E894ED
:10673000A5912591359145915591A6F3EF010E94C0
:10674000A231FE019701A801DA9469F7DF90EF907A
:10675000FF900F911F91CF91DF9108959B01AC01A4
:1067600060E070E080E89FE30C94F7310C94D23045
:106770000C9474340E940231D8F39923C9F3940F16
:10678000511DA3F39150504094F059F0882332F0FA
:10679000660F771F881F91505040C1F79E3F5105EB
:1067A0002CF7880F911D9695879597F908955F3F6F
:1067B000ACF0983E9CF0BB27869577956795B7958A
:1067C00008F4B1609395C1F7BB0F58F711F460FF5F
:1067D000E8CF6F5F7F4F8F4F9F4FE3CF0C941D31FA
:1067E00016F00C9474340C94D83068940C94D23015
:1067F0000E940231A8F39923C1F3AEF3DF93CF9344
:106800001F930F93FF92C92FDD2788232AF021972A
:10681000660F771F881FDAF720E030E040E85FEB73
:106820009FE3883920F0803E38F021968F770E94D0
:106830008B31E0E9F0E004C00E948B31EDEBF0E039
:106840000E9487338B01BE01EC01FB2E6F5771094B
:106850007595771F880B990B0E94033028E132E76A
:1068600041E35FE30E947530AF2D9801AE01FF90C8
:106870000F911F91CF91DF910E94A2310C94E930CA
:10688000FA01DC01AA0FBB1F9B01AC01BF5728F422
:10689000222733274427507820C0B75190F4AB2FDC
:1068A0000024469537952795011CA395D2F3002027
:1068B00071F0220F331F441FB395DAF30ED00C94FE
:1068C0008A3161307105A0E88A07B94630F49B012E
:1068D000AC016627772788279078309621F02083AF
:1068E00031834283538308959F3F31F0915020F4C8
:1068F000879577956795B795880F911D969587959C
:1069000097F90895DB018F939F930E943931BF91CE
:10691000AF91A29F800D911DA39F900DB29F900DEE
:1069200011240895AA1BBB1B51E107C0AA1FBB1F5E
:10693000A617B70710F0A61BB70B881F991F5A950B
:10694000A9F780959095BC01CD01089597FB072E7E
:1069500016F4009407D077FD09D00E94923407FC0A
:1069600005D03EF4909581959F4F0895709561955F
:106970007F4F0895A1E21A2EAA1BBB1BFD010DC07B
:10698000AA1FBB1FEE1FFF1FA217B307E407F507DF
:1069900020F0A21BB30BE40BF50B661F771F881FBB
:1069A000991F1A9469F760957095809590959B0151
:1069B000AC01BD01CF010895EE0FFF1F0590F491CA
:1069C000E02D0994B7FF0C9439310E943931821BB4
:1069D000930B0895DF93CF931F930F939A9DF02D00
:1069E000219FF00D8B9DF00D8A9DE02DF10D039FF1
:1069F000F00D029FE00DF11D4E9DE00DF11D5E9D1D
:106A0000F00D4F9DF00D7F936F93BF92AF925F9308
:106A10004F93D5010E947B318B01AC01D7010E94BD
:106A20007B31EB01E80FF91FD6010E9439352F9118
:106A30003F91D6010E947B31C60FD71FE81FF91F77
:106A4000AF91BF910E9439352F913F910E947B31C8
:106A5000C60FD71FE81FF91FD6010E947B31E60F32
:106A6000F71F9801BE01CF010F911F91CF91DF91C8
:106A700008950E947B31460F571FC81FD91F08F485
:106A800031960895689401C0E894F92FF12B12F023
:106A90000C947635A0E0B0E0E0E5F5E30C944A31E3
:106AA000092E059422F40E94D235112392F4F0E8C5
:106AB0000F26FFEFE094F09400951095B094C094E9
:106AC000D094A194BF0ACF0ADF0AEF0AFF0A0F0B86
:106AD0001F0B0E94813507FC0E94D235CDB7DEB76F
:106AE000ECE00C946631689401C0E8948F929F9218
:106AF000CF93DF930E948135DF91CF919F908F904C
:106B0000089588249924F401E401B0E49F93AA270E
:106B10009A158B049C04ED05FE05CF05D007A1074F
:106B200098F4AD2FDC2FCF2FFE2FE92D982C892E36
:106B3000982F872F762F652F542F432F322F222700
:106B4000B85031F7BF9127C01B2EBF91BB27220F32
:106B5000331F441F551F661F771F881F991F881CEE
:106B6000991CEE1FFF1FCC1FDD1FAA1FBB1F8A141D
:106B70009B04EC05FD05CE05DF05A007B10748F035
:106B80008A189B08EC09FD09CE09DF09A00BB10B9F
:106B900021601A94E1F62EF49401AF01BE01CD01FB
:106BA000000C08956095709580959095309540956E
:106BB000509521953F4F4F4F5F4F6F4F7F4F8F4FF6
:106BC0009F4F0895002E083090F0982F872F762F32
:106BD000652F542F432F322F22270850F4CF220F36
:106BE000331F441F551F661F771F881F991F0A9563
:106BF000B2F7002D089597FD1094002E083098F0FC
:106C00000850232F342F452F562F672F782F892F89
:106C1000912DF4CF1594979587957795679557950E
:106C20004795379527950A95AAF71124002D0895C1
:106C30002A0D3B1D4C1D5D1D6E1D7F1D801F911F6C
:106C400008952A193B094C095D096E097F09800BDB
:106C5000910B08950024A7FD00942A1730054005E4
:106C60005005600570058005900508950F931F93EA
:106C7000CF93DF938230910510F482E090E0E091B1
:106C80001706F091180630E020E0B0E0A0E0309761
:106C900099F42115310509F44AC0281B390B243019
:106CA0003105D8F58A819B816115710589F1FB0158
:106CB00093838283FE0111C040815181028113813F
:106CC00048175907E0F04817590799F4109761F0F1
:106CD00012960C93129713961C933296CF01DF9164
:106CE000CF911F910F9108950093170610931806E6
:106CF000F4CF2115310551F04217530738F0A9019F
:106D0000DB019A01BD01DF01F801C1CFEF01F9CF2D
:106D10009093180680931706CDCFFE01E20FF31F64
:106D2000819391932250310939832883D7CF2091C1
:106D3000150630911606232B41F420911001309155
:106D40001101309316062093150620910E01309103
:106D50000F012115310541F42DB73EB740911201C5
:106D600050911301241B350BE0911506F091160686
:106D7000E217F307A0F42E1B3F0B2817390778F012
:106D8000AC014E5F5F4F2417350748F04E0F5F1F71
:106D90005093160640931506819391939FCFF0E090
:106DA000E0E09CCFCF93DF930097E9F0FC013297AE
:106DB00013821282A0911706B0911806ED0130E0FF
:106DC00020E01097A1F420813181820F931F209140
:106DD0001506309116062817390709F061C0F0939F
:106DE0001606E0931506DF91CF910895EA01CE17BC
:106DF000DF07E8F54A815B819E0141155105B1F736
:106E0000E901FB83EA8349915991C40FD51FEC171F
:106E1000FD0761F4808191810296840F951FE9013D
:106E200099838883828193819B838A83F0E0E0E069
:106E300012968D919C9113970097B9F52D913C91E5
:106E40001197CD010296820F931F20911506309164
:106E500016062817390739F6309751F5109218069B
:106E600010921706B0931606A0931506BCCFD383D5
:106E7000C28340815181840F951FC817D90761F4DF
:106E80004E5F5F4F88819981480F591F518340831E
:106E90008A819B81938382832115310509F0B0CFCC
:106EA000F0931806E09317069ECFFD01DC01C0CFDA
:106EB00013821282D7CFB0E0A0E0E1E6F7E30C94B2
:106EC00046318C01009751F4CB010E9436368C017B
:106ED000C801CDB7DEB7E0E10C946231FC01E60FEA
:106EE000F71F9C0122503109E217F30708F49DC0F7
:106EF000D901CD91DC911197C617D70798F0C5300D
:106F0000D10530F3CE0104978617970708F3C61B07
:106F1000D70B2297C193D1936D937C93CF010E949D
:106F2000D236D6CF5B01AC1ABD0A4C018C0E9D1E29
:106F3000A0911706B0911806512C412CF12CE12C90
:106F4000109731F5809115069091160688159905D0
:106F500009F05CC04616570608F058C080910E0133
:106F600090910F01009741F48DB79EB740911201A7
:106F700050911301841B950BE817F90708F055C0D1
:106F8000F0931606E0931506F90171836083A0CF94
:106F90008D919C91119712966C90129713967C90FC
:106FA0001397A815B90559F56C0142E0C40ED11C20
:106FB000CA14DB0420F1AC014A195B09DA0112960C
:106FC000159780F06282738251834083D9016D935B
:106FD0007C93E114F10471F0D7011396FC93EE93C6
:106FE000129776CF22968C0F9D1FF9019183808393
:106FF000F301EFCFF0931806E093170669CF481618
:10700000590608F42C017D01D3019ACFCB010E94CF
:1070100036367C01009749F0AE01B8010E94203855
:10702000C8010E94D236870153CF10E000E050CF54
:107030009111089581568A5108F480528558089517
:10704000FB01DC0102C001900D9241505040D8F785
:107050000895FB01DC0101900D920020E1F70895F5
:10706000FB01DC014150504030F08D9101908019BE
:1070700019F40020B9F7881B990B0895FB01DC0176
:107080004150504048F001900D920020C9F701C0D6
:107090001D9241505040E0F70895FB015191552356
:1070A000A9F0BF01DC014D9145174111E1F759F4F9
:1070B000CD010190002049F04D9140154111C9F3D7
:1070C000FB014111EFCF81E090E00197089511E0BD
:1070D000CEE4D1E004C0FE010E94DC342196CF341E
:1070E000D107C9F7F894FFCF0000A040C800010104
:1070F00064000000F041000019068000FF018600D6
:1071000000000000795E00BC00770100000000353F
:10711000027C01C2018202F301D101E501000000FD
:1071200000200AF3094F0A2406EC09D909CA09000C
:1071300000000025067C014F0A2406810699060CF2
:10714000060D0A005245420056455200235665720C
:1071500073696F6E3A004C4F4700234C6F67676549
:1071600072204E616D653A0053484F57533D0047BA
:10717000455400732000534156453D0054494D4548
:10718000493D0023496E74657276616C3D00544937
:107190004D45443D00234475726174696F6E3D0036
:1071A00042543D00534C20503D00506120756E6CA0
:1071B000696B656C792100685061004E45543D0053
:1071C00055565A002355562056303D00562000444F
:1071D000535400234453542063616C696272617498
:1071E000656420666F722023004D533D002C002300
:1071F000496E636F727265637421204D533D313265
:107200003344334435005428312C322C33293D008B
:10721000206F4320445320546865726D6F6D657410
:1072200065720020572F6D5E3200555620496E74EE
:10723000656E7369747900572F6D5E322000555664
:107240003D0070706D00434F323D00206E672F4C43
:1072500000504D28312E302C322E352C3130293D26
:107260000068506120006F430020413D004C696779
:10727000687420496E74656E7369747900206C7847
:1072800020004C3D00495220466C616D65204C65E4
:1072900076656C3D00476173206C6576656C3D00DA
:1072A000204D756C746973656E736F72730023453E
:1072B0006E61626C65002344697361626C650044B1
:1072C000440023496E76616C6964206B6579210006
:1072D000424E4D4C3033006E616E6F42326936441F
:1072E00053546300234E6F2053656E736F722100F9
:1072F00057656C636F6D653A0023626D702066613F
:10730000696C65640073657269616C3A20002D35A3
:08731000002D34002D330000B4
:107E0000112484B714BE81FFF0D085E080938100F7
:107E100082E08093C00088E18093C10086E0809377
:107E2000C20080E18093C4008EE0C9D0259A86E02C
:107E300020E33CEF91E0309385002093840096BBD3
:107E4000B09BFECF1D9AA8958150A9F7CC24DD24C4
:107E500088248394B5E0AB2EA1E19A2EF3E0BF2EE7
:107E6000A2D0813461F49FD0082FAFD0023811F036
:107E7000013811F484E001C083E08DD089C08234E0
:107E800011F484E103C0853419F485E0A6D080C0E4
:107E9000853579F488D0E82EFF2485D0082F10E0AE
:107EA000102F00270E291F29000F111F8ED06801E7
:107EB0006FC0863521F484E090D080E0DECF843638
:107EC00009F040C070D06FD0082F6DD080E0C81688
:107ED00080E7D80618F4F601B7BEE895C0E0D1E017
:107EE00062D089930C17E1F7F0E0CF16F0E7DF06D8
:107EF00018F0F601B7BEE89568D007B600FCFDCFD4
:107F0000A601A0E0B1E02C9130E011968C91119780
:107F100090E0982F8827822B932B1296FA010C0160
:107F200087BEE89511244E5F5F4FF1E0A038BF0790
:107F300051F7F601A7BEE89507B600FCFDCF97BE46
:107F4000E89526C08437B1F42ED02DD0F82E2BD052
:107F50003CD0F601EF2C8F010F5F1F4F84911BD097
:107F6000EA94F801C1F70894C11CD11CFA94CF0C13
:107F7000D11C0EC0853739F428D08EE10CD085E9AC
:107F80000AD08FE07ACF813511F488E018D01DD067
:107F900080E101D065CF982F8091C00085FFFCCF94
:107FA0009093C60008958091C00087FFFCCF809118
:107FB000C00084FD01C0A8958091C6000895E0E648
:107FC000F0E098E1908380830895EDDF803219F02E
:107FD00088E0F5DFFFCF84E1DECF1F93182FE3DFCA
:107FE0001150E9F7F2DF1F91089580E0E8DFEE27F6
:047FF000FF270994CA
:027FFE00040479
:00000001FF
